:10000000A2C20000D1C20000CFC20000CDC20000D9
:10001000CBC20000C9C20000C7C20000C5C20000B8
:10002000C3C20000C1C20000BFC20000BDC20000C8
:10003000BBC20000B9C20000B7C20000B5C20000D8
:10004000B3C200000C94D42AAFC20000ADC20000BD
:100050000C94612DA9C20000A7C200000C94802955
:10006000A3C200000C94A3270C947A279DC2000021
:100070009BC2000099C2000097C2000095C2000018
:100080000C94A72A91C200008FC200008DC200000C
:100090008BC2000089C2000087C2000085C2000038
:1000A00083C2000081C200000C947A2A7DC2000045
:1000B0007BC2000079C2000077C200000C944D2A78
:1000C00073C2000071C200006FC200006DC2000068
:1000D0006BC2000069C2000067C2000065C2000078
:1000E00063C20000E002ED02F602FF020C031503FA
:1000F000B106B106B106B106B10622032F033C03D7
:10010000B106490352035B03680371037A03830357
:100110008C039503B1069E03A703B003B106B10695
:10012000B106B903C203CB03B106B106D403E103A0
:10013000B106B106B106EE03FB030804B1061504CF
:100140001E042704B106B106B10630043904420486
:10015000B1064F045C046904B106B106B106760429
:1001600083049004B1069D04AA04B704B106B10645
:10017000B106C404D104DE04B106EB04F404FD04AA
:10018000B106B106B106B106B106B106B106B106B7
:10019000B106B106B106B106B106B106B106B106A7
:1001A000B106B106B106B106B106B106B106210528
:1001B0002A053305B1063C0545054E05B106B106D5
:1001C000B106570564057105B1067E058B059805D6
:1001D000B106B106B106A505B205BF05B106CC054D
:1001E000D505DE05B106B106B106E705F005F9054E
:1001F000B106B106B106B106B106B106B106B10647
:10020000B106B106B10606050F051805B106B1061F
:10021000B106B106B106B106B106B106B106B10626
:10022000B106B106B106B106B106B106B106B10616
:10023000B106B106B106B106B106B106B106B10606
:10024000B106B106B106B106B106B106B106B106F6
:10025000B106B106B106B106B106B106B106B106E6
:10026000B106B106B106B106B106B106B106B106D6
:10027000B106B106B10602060B061806B106250640
:100280002E063B06B106B106B106480651065E06CB
:10029000B1066B0674068106B106B106B1068E067C
:1002A0009706A406760A7B0A800A8A0A940A0D0B2E
:1002B0009E0AA60AAE0AB80AC20ACC0ADB0AE50AF6
:1002C0000D0BEF0AF90A030BD425D725C625CA253D
:1002D000D0250E26DB25DF25E525E925ED25F325AF
:1002E000F725FB250E260126052609264E414E49F7
:1002F0004E495459494E46CDCCCC3D0AD7233C17E4
:10030000B7D13877CC2B329595E6241FB14F0A0030
:100310000020410000C84200401C4620BCBE4CCA20
:100320001B0E5AAEC59D7400407A10F35A00A0729D
:100330004E18090010A5D4E80000E8764817000020
:10034000E40B54020000CA9A3B000000E1F50500EE
:100350000080969800000040420F000000A0860137
:10036000000000102700000000E803000000006407
:1003700000000000000A0000000000010000000072
:10038000002C76D888DC674F0823DFC1DFAE59E147
:10039000B1B796E5E3E453C63AE651997696E8E6B6
:1003A000C28426EB898C9B62ED407C6FFCEFBC9C89
:1003B0009F40F2BAA56FA5F490055A2AF75C936B9B
:1003C0006CF9676DC11BFCE0E40D47FEF520E6B556
:1003D00000D0ED902E0300943577050080841E0830
:1003E0000000204E0A000000C80C333333330F984E
:1003F0006E12831141EF8D2114893BE65516CFFE15
:10040000E6DB18D1844B381BF77C1D901DA4BBE4A0
:1004100024203284725E228100C9F124ECA1E53DE2
:100420002700000A0B02090C0D0E08070304010047
:1004300000000000000000000000000000000000BC
:100440000000000000000000000000000012111079
:10045000000000000000000000000000000000009C
:100460000000000000000000002100240027002AF6
:10047000002D003000330001010000040107010AD3
:100480000100002200250028002B002E003100343E
:100490000002010000050108010B010000200023FB
:1004A00000260029002C002F00320000010000036C
:1004B00001060109010505050507050808080802E8
:1004C0000202020A0A0808040404040101010101ED
:1004D0000101010303030303030303040707070CDC
:1004E0000C0C0C0C0C0C0C02020202060606060692
:1004F0000606060B0B0B0B0B0B0B0B01021020203F
:100500000808102040102040800201020108040267
:1005100001010204081020408080402010080402DD
:100520000180040201804020100804020108040236
:10053000010102040810204080010204081020403C
:1005400080005B46564611241FBECFEFD1E2DEBFCE
:10055000CDBF00E00CBF17E0A0E0B2E0E4EBF0EAB2
:1005600000E00BBF02C007900D92A234B107D9F78B
:100570002CE0A2E4B7E001C01D92AC3EB207E1F767
:1005800012E0C2EAD2E000E006C021970109802F04
:10059000FE010E943D4FC13AD10780E00807A9F74C
:1005A0000E944C3C0C9449502BCD603E710508F0E4
:1005B000D8C3FB018827EE58FF4F8F4F0C943D4F57
:1005C00081E090E0A0E0B0E0809356079093570759
:1005D000A0935807B0935907089510925A071092A4
:1005E0005B0710925C0710925D07089510925E07FA
:1005F00010925F071092600710926107089581E0E2
:1006000090E0A0E0B0E08093620790936307A0932E
:100610006407B09365070895109266071092670704
:100620001092680710926907089583E090E0A0E0B7
:10063000B0E080936A0790936B07A0936C07B09328
:100640006D07089588E790E0A0E0B0E0809382070E
:1006500090938307A0938407B0938507089588E754
:1006600090E0A0E0B0E08093860790938707A09386
:100670008807B0938907089588E790E0A0E0B0E08C
:1006800080938A0790938B07A0938C07B0938D0774
:100690000895109292071092930710929407109267
:1006A0009507089510929607109297071092980751
:1006B00010929907089581E090E0A0E0B0E0809367
:1006C0009A0790939B07A0939C07B0939D0708956A
:1006D00010929E0710929F071092A0071092A107F8
:1006E00008951092A2071092A3071092A4071092E7
:1006F000A50708951092A6071092A7071092A807C1
:100700001092A90708951092AA071092AB071092B1
:10071000AC071092AD0708951092AE071092AF0784
:100720001092B0071092B10708951092B20710927C
:10073000B3071092B4071092B50708951092BA0744
:100740001092BB071092BC071092BD07089510923B
:10075000BE071092BF071092C0071092C1070895FC
:100760001092C2071092C3071092C4071092C507D7
:1007700008951092D2071092D3071092D4071092C6
:10078000D50708951092D6071092D7071092D80770
:100790001092D90708951092DA071092DB07109291
:1007A000DC071092DD07089581E090E0A0E0B0E062
:1007B0008093E6079093E707A093E807B093E907D3
:1007C000089581E090E0A0E0B0E08093EA07909384
:1007D000EB07A093EC07B093ED0708958CE291E04E
:1007E000A0E0B0E08093FA079093FB07A093FC078A
:1007F000B093FD0708958CE291E0A0E0B0E0809313
:10080000FE079093FF07A0930008B0930108089596
:100810008CE291E0A0E0B0E080930208909303089E
:10082000A0930408B0930508089510920A08109246
:100830000B0810920C0810920D08089510920E08E3
:1008400010920F081092100810921108089510923B
:1008500012081092130810921408109215080895A7
:100860001092220810922308109224081092250852
:1008700008951092260810922708109228081092C6
:100880002908089581E090E0A0E0B0E080932A0874
:1008900090932B08A0932C08B0932D08089585E021
:1008A00090E0A0E0B0E08093320890933308A093EA
:1008B0003408B0933508089585E090E0A0E0B0E0FA
:1008C0008093360890933708A0933808B09339087E
:1008D000089589E190E0A0E0B0E080933A08909319
:1008E0003B08A0933C08B0933D08089582E390E054
:1008F000A0E0B0E080934A0890934B08A0934C0886
:10090000B0934D08089582E390E0A0E0B0E08093BA
:100910004E0890934F08A0935008B0935108089543
:1009200082E390E0A0E0B0E08093520890935308F7
:10093000A0935408B0935508089582E390E0A0E096
:10094000B0E080935A0890935B08A0935C08B09342
:100950005D08089582E390E0A0E0B0E080935E0837
:1009600090935F08A0936008B0936108089582E3B4
:1009700090E0A0E0B0E08093620890936308A093B9
:100980006408B0936508089580E991E0A0E0B0E0C4
:100990008093720890937308A0937408B0937508BD
:1009A000089580E991E0A0E0B0E08093760890930C
:1009B0007708A0937808B0937908089580E991E0CA
:1009C000A0E0B0E080937A0890937B08A0937C0825
:1009D000B0937D08089510928208109283081092B7
:1009E000840810928508089510928608109287084E
:1009F0001092880810928908089510928A0810921F
:100A00008B0810928C0810928D08089510929A0904
:100A100010929B0910929C0910929D0908951092C2
:100A20009E0910929F091092A0091092A1090895A1
:100A30001092A2091092A3091092A4091092A5097C
:100A400008951092EA081092EB081092EC081092A8
:100A5000ED0808951092EE081092EF081092F00839
:100A60001092F10808951092F2081092F308109273
:100A7000F4081092F50808951092FA081092FB08F5
:100A80001092FC081092FD0808951092FE08109232
:100A9000FF081092000910920109089510920209AE
:100AA000109203091092040910920509089585E037
:100AB00090E0A0E0B0E08093120990931309A09316
:100AC0001409B0931509089585E090E0A0E0B0E026
:100AD0008093160990931709A0931809B0931909E8
:100AE000089585E090E0A0E0B0E080931A0990932B
:100AF0001B09A0931C09B0931D09089584EB95E18F
:100B0000A0E0B0E08093220990932309A0932409E8
:100B1000B0932509089584EB95E1A0E0B0E08093BF
:100B2000260990932709A0932809B09329090895CD
:100B300084EB95E1A0E0B0E080932A0990932B0923
:100B4000A0932C09B0932D09089585E090E0A0E0D2
:100B5000B0E080933A0990933B09A0933C09B0938D
:100B60003D09089585E090E0A0E0B0E080933E0963
:100B700090933F09A0934009B0934109089585E0FF
:100B800090E0A0E0B0E08093420990934309A093E5
:100B90004409B0934509089510924A0910924B09EF
:100BA00010924C0910924D09089510924E0910921E
:100BB0004F0910925009109251090895109252094C
:100BC00010925309109254091092550908951092E9
:100BD00062091092630910926409109265090895E0
:100BE00010926609109267091092680910926909BB
:100BF000089510926A0910926B0910926C09109274
:100C00006D09089510927A0A10927B0A10927C0A5C
:100C100010927D0A08958CE390E0A0E0B0E080930C
:100C20007E0A90937F0AA093800AB093810A089568
:100C300081E090E0A0E0B0E08093820A9093830A84
:100C4000A093840AB093850A089510928A0A10929C
:100C50008B0A10928C0A10928D0A08958CE390E012
:100C6000A0E0B0E080938E0A90938F0AA093900A40
:100C7000B093910A089581E090E0A0E0B0E0809305
:100C8000920A9093930AA093940AB093950A0895B8
:100C90001092A20A1092A30A1092A40A1092A50A16
:100CA00008958CE390E0A0E0B0E08093A60A9093D2
:100CB000A70AA093A80AB093A90A089581E090E03A
:100CC000A0E0B0E08093AA0A9093AB0AA093AC0A8C
:100CD000B093AD0A08951092B20A1092B30A10921E
:100CE000B40A1092B50A08958CE390E0A0E0B0E059
:100CF0008093B60A9093B70AA093B80AB093B90A42
:100D0000089581E090E0A0E0B0E08093BA0A90936B
:100D1000BB0AA093BC0AB093BD0A08951092CA0AF8
:100D20001092CB0A1092CC0A1092CD0A08958CE34F
:100D300090E0A0E0B0E08093CE0A9093CF0AA09319
:100D4000D00AB093D10A089581E090E0A0E0B0E02D
:100D50008093D20A9093D30AA093D40AB093D50A71
:100D60000895660F771F660F771FFB01EA5AF84F49
:100D7000108211821282138208950F931F93CF93D2
:100D8000DF938C01C0E0D0E0BE01C8010E94EF32C9
:100D9000882319F0BE01C80108DC2196C13ED105A7
:100DA00099F7DF91CF911F910F9108954F925F9224
:100DB0006F927F928F929F92AF92BF92CF92DF926B
:100DC000EF92FF92CF93DF935B01EB01CC0FDD1F1E
:100DD000CE010E94C44D482E512C612C712CCE01A5
:100DE00001960E94C44DC82ED12CE12CF12C8DE827
:100DF000A81AB10883E0A816B10488F5CE0144967C
:100E00000E94C44D882E912CA12CB12CCE01459668
:100E10000E94C44D482F50E060E070E08FEF8816CC
:100E20009104A104B104A9F44F3F51056105710576
:100E300081F48FEF481651046104710481F48FEF3F
:100E4000C816D104E104F10451F46FEF7FEFCB0138
:100E50002BC040385105610571056CF0F6CF80E874
:100E6000C816D104E104F10484F740E050E0BA016F
:100E7000812C912C5401FE2CED2CDC2CCC24C40CA8
:100E8000D51CE61CF71C540199248824C80CD91CD5
:100E9000EA1CFB1C742F662755274427CB01BA0197
:100EA0006C0D7D1D8E1D9F1DDF91CF91FF90EF90EA
:100EB000DF90CF90BF90AF909F908F907F906F907A
:100EC0005F904F9008950C9496470C9496470C941D
:100ED0009647CF93DF93EB0120E030E040E85FE3FB
:100EE0006A817B818C819D810E94A84C811113C0F5
:100EF0008DE994E00E94053B0E94DD16FC01E25B57
:100F0000FF4F1082118212821382E05DFE4F108A21
:100F1000118A128A138A20E030E040E85FE36E8194
:100F20007F81888599850E94A84C811113C08DEA24
:100F300094E00E94053B0E94DD16FC01E853FF4F40
:100F40001082118212821382EE52FF4F108A118A90
:100F5000128A138A20E030E040E85FE36A857B85EF
:100F60008C859D850E94A84C811113C08DEB94E067
:100F70000E94053B0E94DD16FC01EE5BFE4F1082D5
:100F8000118212821382EC58FF4F108A118A128A42
:100F9000138A0E9489180E94931780E090E0DF91E5
:100FA000CF9108950F93CF93DF938091860B81119A
:100FB0007BC081E08093860B0E94DD16EC0103B1BB
:100FC00023B14091000160910001001F0027001F24
:100FD000221F2227221F41706695617082589E4F02
:100FE0000E94843503B123B140B160B1001F0027D6
:100FF000001F221F2227221F42FB442740F966952B
:101000006170CE0186569E4F0E94843503B123B194
:1010100040B160B1001F0027001F221F2227221F9E
:1010200046FB442740F9661F6627661FCE018A5497
:101030009E4F0E948435FE01E159FF4F8081882335
:1010400061F0709780819181A281B3810196A11D89
:10105000B11D80839183A283B383FE01E751FF4FCB
:101060008081882361F0709780819181A281B38112
:101070000196A11DB11D80839183A283B383FE01DC
:10108000ED59FE4F8081882369F0CD5ADE4F88816B
:101090009981AA81BB810196A11DB11D8883998385
:1010A000AA83BB831092860BDF91CF910F91089595
:1010B0008F929F92AF92BF92CF92DF92EF92FF9268
:1010C0000F931F930E94DD1621E02F931F921F9212
:1010D0001F921F92812C912CA12CB12CC12CD12CB0
:1010E000760197018601B701A601A4D20F900F9057
:1010F0000F900F900F9080E090E01F910F91FF9064
:10110000EF90DF90CF90BF90AF909F908F90089519
:10111000EF92FF920F931F93CF93DF9300D01F9214
:10112000CDB7DEB78B017B01EE0CFF1C622FC70130
:1011300029833A834B835C830E94CC4D29813A8179
:101140004B815C81992757FD9A95852F742F632FCA
:10115000C70101960E94CC4D0D58110929813A8191
:101160004B815C8103301105A8F4BA01992777FD02
:101170009095892FC70144960E94CC4D29813A81D0
:101180004B815C81652F772788279927C701459672
:101190000E94CC4D80E090E00F900F900F900F9048
:1011A000DF91CF911F910F91FF90EF900895CF9213
:1011B000DF92EF92FF92CF93DF93EB010E94EF3229
:1011C000882359F1FE01EE0FFF1FEE0FFF1FEA5AB1
:1011D000F84FC080D180E280F3808DEC94E00E94D3
:1011E000053B8EE496E00E94053B81ED94E00E9471
:1011F000053BCE010E94783B8EE496E00E94053BC1
:1012000083ED94E00E94053BC701B6010E94513B6B
:101210000E9489180E94931704C085ED94E00E94F3
:10122000053B80E090E0DF91CF91FF90EF90DF9061
:10123000CF900895EF92FF920F931F93CF93DF9378
:101240008091870B9091880B892B09F066C084E010
:1012500090E00E940147EC0160E070E0A7DD161607
:101260001706FCF0CE0189DD96E5E92E97E0F92E10
:1012700000E010E0B801CE010E94EF32882341F077
:10128000F7012081318142815381B801CE0140DFD5
:101290000F5F1F4FF4E0EF0EF11C0639110551F7F7
:1012A00038C063E070E0CE0181DD613071058105F9
:1012B000910569F586E5E82E87E0F82E00E010E05C
:1012C000B801CE010E94EF328823C1F0B801CE01EF
:1012D0006DDDF70160837183828393836F3F7F4F5E
:1012E0008F4F9F4F59F4B801CE015FD9F70120818C
:1012F000318142815381B801CE010ADF0F5F1F4F58
:10130000F4E0EF0EF11C013E1105D1F602C0CE0152
:1013100034DDD093880BC093870B8091870B90911D
:10132000880BDF91CF911F910F91FF90EF9008955F
:10133000089508950895EF92FF920F931F93CF930E
:10134000DF93162F072F7A014115510559F4862F87
:101350000E94D92731E020E0019709F030E0C32F47
:10136000D22F26C04130510509F5262F663310F0E3
:101370002AEC260F80917B00922F9870877F892B13
:1013800080937B002770206420937C0080917A00FA
:10139000806480937A0080917A0086FDFCCFC091B2
:1013A000780080917900D0E0D82B02C0C0E0D0E076
:1013B00082E0E816F10410F587EF94E00E94053B07
:1013C0008EE496E00E94053B81ED94E00E94053B8F
:1013D000812F902F0E94783B8EE496E00E94053B7F
:1013E00083ED94E00E94053BCE010E94783B0E9471
:1013F00089180E94931780E090E002C081E090E09D
:10140000DF91CF911F910F91FF90EF9008958BEF97
:1014100094E00E94053B0E9489180E94D01A0E9405
:1014200089180E94A5170E94A53440E050E068E0AA
:1014300070E081DF0E94A53440E050E069E070E098
:101440007ADF0E94A53440E050E06AE070E073DF8C
:101450000E94A53440E050E06DE070E06CDF80E079
:1014600090E008950F931F93CF93DF938B01EA01D0
:10147000AB01415051094433510508F0D4C022302A
:10148000310508F0D0C048E3429FF001439FF00DC2
:101490001124E60FF71FE80FF91F81E08083232B4B
:1014A00011F46C2F07C061E0802F0E94F52820976F
:1014B00039F460E0802F0E94012880E090E0B5C000
:1014C000CF3FD10509F4ADC0F801EF5DFB4FE491CA
:1014D0008E2F90E0FC013197E231F10508F09DC0BC
:1014E0008827EE5AFE4F8F4F0C943D4F84B580688D
:1014F00084BDC7BDE2CF84B5806284BDC8BDDDCFE9
:1015000080918000806880938000D0938900C09390
:101510008800D3CF80918000806280938000D09338
:101520008B00C0938A00C9CF80918000886080932F
:101530008000D0938D00C0938C00BFCF8091B0000D
:1015400080688093B000C093B300B7CF8091B000A3
:1015500080628093B000C093B400AFCF80919000C0
:10156000806880939000D0939900C0939800A5CF95
:1015700080919000806280939000D0939B00C093F4
:101580009A009BCF80919000886080939000D093C8
:101590009D00C0939C0091CF8091A00080688093B3
:1015A000A0008091A0008F7B8093A000D093A90021
:1015B000C093A80082CF8091A00080628093A00099
:1015C000D093AB00C093AA0078CF8091A000886030
:1015D0008093A000D093AD00C093AC006ECF8091FB
:1015E0002001806880932001D0932901C0932801B5
:1015F00064CF80912001806280932001D0932B01E1
:10160000C0932A015ACF80912001886080932001E5
:10161000D0932D01C0932C0150CFC038D1050CF4CC
:1016200048CF61E047CF81E090E0DF91CF911F91FB
:101630000F9108952F923F924F925F926F927F92F7
:101640008F929F92AF92BF92CF92DF92EF92FF92D2
:101650000F931F93CF93DF93CDB7DEB7E6970FB607
:10166000F894DEBF0FBECDBF1C012A013B010B87E2
:101670001C872D873E872E960EAD1FAD2E97FC0141
:10168000E55AFD4F60817181828193810E94AE4C49
:101690009B01AC01C301B2010E940D4D0E94044F99
:1016A0006B8B7C8B8D8B9E8BF101E15AFD4F6081A2
:1016B0007181828193810E94AE4C9B01AC016B854C
:1016C0007C858D859E850E940D4D0E94044F6B8FF9
:1016D0007C8F8D8F9E8FF101ED59FD4F608171815F
:1016E000828193810E94AE4C9B01AC01C701B6017F
:1016F0000E940D4D0E94044F6F8F78A389A39AA377
:101700000E9474296B877C878D879E87F101E45244
:10171000FE4F118210823296118210823E96A114E1
:10172000B10461F0C501A0E0B0E040815181628167
:10173000738184179507A607B70714F0A080B180BE
:10174000F101E051FE4F8114910461F0C401A0E069
:10175000B0E0408151816281738184179507A607AB
:10176000B70714F080809180F101EC50FE4F011515
:10177000110561F0C801A0E0B0E0408151816281B3
:10178000738184179507A607B70714F000811181AC
:10179000310120E1620E711CC501A0E0B0E0F10151
:1017A00080A791A7A2A7B3A72101FAE84F0E511C69
:1017B000A12CB12CD20158968D929D92AD92BC92E3
:1017C0005B974101BCEF8B1ABEEF9B0A20E030E033
:1017D000F401008F118F228F338F0E9489180E948D
:1017E00089180E9489180E94891840914A075091CF
:1017F0004B0760914C0770914D074BAB5CAB6DABE9
:101800007EAB0E94891880914E0790914F07A0915E
:101810005007B09151078F87988BA98BBA8B0E9484
:101820008918A0905207B0905307C0905407D090E9
:101830005507F101E959FD4F10821182128213827E
:101840003496108211821282138234961082118291
:101850001282138234961182108232961182108283
:1018600032961182108232964BA95CA96DA97EA98D
:10187000408351836283738334968F859889A989C5
:10188000BA8980839183A283B3833496A082B18284
:10189000C282D3822F96EFAC2F970B891C892D899A
:1018A0003E89C3010E941A2E8823F9F085E393E054
:1018B0000E94053B8AEA94E00E94053BF101EE5A42
:1018C000FF4F6081718182819381E75FFD4F2081AD
:1018D0003181428153810E94DA4DCA01B9010E94CF
:1018E000513B0E9489180E9493176096EFAC609755
:1018F0000B8D1C8D2D8D3E8D4F85588969897A8978
:10190000C2010E941A2E8823F9F081E393E00E941D
:10191000053B8AEB94E00E94053BF101E453FF4F45
:101920006081718182819381ED56FE4F20813181EA
:10193000428153810E94DA4DCA01B9010E94513B94
:101940000E9489180E9493176196EFAC61970F8DE2
:1019500018A129A13AA1B601A501C4010E941A2E1D
:101960008823F9F08DE293E00E94053B8AEC94E035
:101970000E94053BF101EA5BFE4F6081718182812B
:101980009381E35EFE4F20813181428153810E9429
:10199000DA4DCA01B9010E94513B0E9489180E9488
:1019A0009317D10151961C92F101E557FF4F108218
:1019B000E658FF4F1082C1010E94562CC1010E94BF
:1019C0005A2CC3010E946832C2010E946832C401CD
:1019D0000E946832F101ED51FE4FFCA3EBA381E0C0
:1019E00090E0918380837101FBE1EF1AFEEFFF0A23
:1019F000D7018D939C93810109511E4FF80191836A
:101A0000808341E050E0B301C1010E94E118D70199
:101A10004D915C91B201C1010E94E118F801408131
:101A20005181B401C1010E94E11811E0F101EE53AE
:101A3000FD4F1083C3010E94072EC2010E94072E92
:101A4000C4010E94072E64E670E080E090E00E94EE
:101A50003C29C10180529E4FDC011C9311961C93BE
:101A6000A1014E515E4FFA0110832F96FFAD2F97C3
:101A7000F1110FC060962FAD6097211105C06196DE
:101A80003FAD6197332339F1910121593F4FF9015E
:101A900010826096FFAD6097F11105C0910127514A
:101AA0003F4FF90110826196FFAD6197F11105C0BA
:101AB00091012D593E4FF90110822F962FAD2F978E
:101AC000FC01208360963FAD60973C936196EFAD3B
:101AD0006197DA01EC93C3010E94C32FC2010E94F7
:101AE000C32FC4010E94C32FC3010E94192FC2013A
:101AF0000E94192FC4010E94192F0E948918DC012D
:101B00001C968C918F87A12CB12CF101E052FE4FD5
:101B1000FC8BEB8B91012F513E4F3C8F2B8FA10102
:101B20004E515E4F58A34F8FC1018D519E4F9CA7C0
:101B30008BA7D101AB51BE4FBEA7ADA73796F8AB6F
:101B4000EFA72F5631403AA729A74F535F4F5AAB03
:101B500049AB8B5191409EA38DA3A35AB109B8A75D
:101B6000AFA3EB89FC89808181110BC0AB8DBC8D4B
:101B70008C91811106C0EF8DF8A18081882309F432
:101B80005DC3FF85F1115AC34BA55CA5B301C1012B
:101B90000E9438194DA55EA5B201C1010E943819F5
:101BA0004FA558A9B401C1010E943819C3010E9470
:101BB000832FC2010E94832FC4010E94832FE9A5B5
:101BC000FAA58081882321F1C3010E94C32FA9A90E
:101BD000BAA98C918823C9F06101B9E6CB1ABDEF8F
:101BE000DB0A7101EEE4EE1AEDEFFE0A81010B57FC
:101BF0001D4F910127583D4FA10149595D4FB1013A
:101C000062587E4FC3010E949A2BA9A5BAA51C92C7
:101C1000F101E451FF4F8081882331F1C2010E941C
:101C2000C32FF101EC55FD4F80818823C9F061017C
:101C3000B5E6CB1ABDEFDB0A7101ECE4EE1AEDEF6D
:101C4000FE0A810107571D4F910123583D4FA10105
:101C500045595D4FB10166567E4FC2010E949A2BD5
:101C6000F101E451FF4F1082F101EA59FE4F8081EA
:101C7000882331F1C4010E94C32FF101EB55FD4FC0
:101C800080818823C9F06101F1E6CF1AFDEFDF0AF8
:101C900071012AE4E21A2DEFF20A810103571D4F68
:101CA00091012F573D4FA10141595D4FB1016A5438
:101CB0007E4FC4010E949A2BF101EA59FE4F108217
:101CC000810101591F4FD8018C91882309F43FC02D
:101CD000F101EF56FD4F60817181072E000C880BDA
:101CE000990B0E94AE4C9B01AC01F101E959FD4FEB
:101CF00060817181828193810E94354F18163CF575
:101D0000D8011C9264E274E081010E521E4FC8019A
:101D10000E94282760E475E0C8010E9428276CE92A
:101D200073E0C8010E9428272F96BFAD2F97BB23D1
:101D300009F473C3F101E258FE4F108A118A128A26
:101D4000138AE053F14010821182128213828101C2
:101D500007511F4FF8018081882309F43FC0E655E1
:101D6000FE4F60817181072E000C880B990B0E9439
:101D7000AE4C9B01AC01F101E559FD4F60817181D1
:101D8000828193810E94354F181644F5F801108224
:101D900064E274E081010E521E4FC8010E942827A0
:101DA00068E675E0C8010E9428276CE973E0C80165
:101DB0000E9428276096FFAD6097FF2309F431C386
:101DC000F101E656FE4F108A118A128A138AADA1DC
:101DD000BEA11D921D921D921C92139781010D5957
:101DE0001E4FF8018081882309F43FC0EE5CFE4F4E
:101DF00060817181072E000C880B990B0E94AE4CFC
:101E00009B01AC01F101E159FD4F6081718182813B
:101E100093810E94354F181644F5D8011C9264E254
:101E200074E081010E521E4FC8010E94282760E90C
:101E300075E0C8010E9428276CE973E0C8010E9480
:101E400028276196BFAD6197BB2309F4EEC2F1016B
:101E5000EA54FE4F108A118A128A138AAFA1B8A5DC
:101E60001D921D921D921C92139760E0C3010E9467
:101E7000922E882369F0F101E25BFF4F10821182FC
:101E800012821382E05DFE4F108A118A128A138A31
:101E900060E0C2010E94922E882369F0EDA1FEA1AC
:101EA0001082118212821382F101E656FE4F108ACF
:101EB000118A128A138A60E0C4010E94922E88233C
:101EC00071F0AFA1B8A51D921D921D921C9213979F
:101ED000F101EA54FE4F108A118A128A138AF10125
:101EE000E159FF4F8081EB89FC898083F101E75143
:101EF000FF4F8081AB8DBC8D8C93E658FF4F808166
:101F0000EF8DF8A18083F101E25BFF4F20813181E9
:101F1000428153812F83388749875A87ADA1BEA15B
:101F20004D915D916D917C91EFA1F8A5C080D1801C
:101F3000E280F3804BAB5CAB6DAB7EAB0E9489184B
:101F40008F819885A985BA8580934A0790934B071E
:101F5000A0934C07B0934D070E9489184BA95CA928
:101F60006DA97EA940934E0750934F076093500789
:101F7000709351070E948918C0925207D09253075C
:101F8000E0925407F0925507C1010E94562CAB898C
:101F9000BC898C91882309F44AC00E9474292B853E
:101FA0003C854D855E85621773078407950760F44D
:101FB0000E9474292B853C854D855E8562177307C9
:101FC00084079507A0F51EC00E9474296B017C014F
:101FD0002B853C854D855E85C21AD30AE40AF50A35
:101FE000F101E15BFD4F2081318142815381A8EEF7
:101FF000B3E00E94F64D6C157D058E059F0508F433
:1020000018C2D6CF0E9474296B017C01F101E15BFB
:10201000FD4F2081318142815381A8EEB3E00E94BF
:10202000F64D6C157D058E059F0508F402C2AB8D3B
:10203000BC8D8C91882309F44AC00E9474292B8599
:102040003C854D855E85621773078407950760F4AC
:102050000E9474292B853C854D855E856217730728
:1020600084079507A0F51EC00E9474296B017C01AE
:102070002B853C854D855E85C21AD30AE40AF50A94
:10208000F101ED5AFD4F2081318142815381A8EE4B
:10209000B3E00E94F64D6C157D058E059F0508F492
:1020A000DEC1D6CF0E9474296B017C01F101ED5A8B
:1020B000FD4F2081318142815381A8EEB3E00E941F
:1020C000F64D6C157D058E059F0508F4C8C1AF8DD2
:1020D000B8A18C91882309F44AC00E9474292B85E9
:1020E0003C854D855E85621773078407950760F40C
:1020F0000E9474292B853C854D855E856217730788
:1021000084079507A0F51EC00E9474296B017C010D
:102110002B853C854D855E85C21AD30AE40AF50AF3
:10212000F101E95AFD4F2081318142815381A8EEAE
:10213000B3E00E94F64D6C157D058E059F0508F4F1
:10214000A4C1D6CF0E9474296B017C01F101E95A28
:10215000FD4F2081318142815381A8EEB3E00E947E
:10216000F64D6C157D058E059F0508F48EC188EA35
:102170009BE00E94E4241816190674F588EA9BE097
:102180000E94C2248F7D8534910531F562E075E0AF
:10219000C1018E529E4F0E94282782E693E00E9442
:1021A000053BB7D7C0D6F101E159FF4F1082E65881
:1021B000FF4F1082E658FF4F1082AB89BC891C92FA
:1021C000EB8DFC8D1082AF8DB8A11C92B1E0BF8762
:1021D000AA24A394B12C03C0A114B10481F067E137
:1021E00075E0C1018E529E4F0E942827EB89FC8921
:1021F0001082AB8DBC8D1C92EF8DF8A11082C101B5
:102200000E94BB3AF101E252FE4F8081918101961A
:10221000918380838D3291400CF4A3CCD101AA52DA
:10222000BE4F8D919C911197892B09F09ACC1496F1
:102230008D919C91892B09F43EC193CC81010A5266
:102240001E4FD8018D919C91892B21F0C1010E94D4
:10225000BB3AF7CF87E295E00E94053B2F96BFADD2
:102260002F97BB23E9F0A114B104D1F4EF85E1115C
:102270003AC08DE193E00E94053B4BD754D660965F
:10228000FFAD6097FF2351F189E193E00E94053B88
:1022900040D749D661962FAD6197211118C023C050
:1022A00060963FAD6097332339F0A114B10421F457
:1022B0004F85411118C0E8CF61965FAD61975523F6
:1022C00091F0A114B10479F48F8581110CC085E1DE
:1022D00093E00E94053B1DD726D605C06196EFAD61
:1022E0006197E111F4CF85E090E0ABA1BCA18D93A3
:1022F0009C9391012B513E4F3C872B87D9018D93A5
:102300009C93810109511E4FF8019183808345E020
:1023100050E0B301C10155D7AB85BC854D915C91AF
:10232000B201C1014ED7F80140815181B401C10110
:1023300048D7C1010E945E2CF101E25BFF4F408152
:10234000518162817381E658FF4F80819181A28122
:10235000B3818F8B988FA98FBA8FE658FF4FC080BB
:10236000D180E280F3804BAB5CAB6DAB7EABD1D662
:102370004BA95CA96DA97EA940934A0750934B07CE
:1023800060934C0770934D07C4D62F89388D498DC3
:102390005A8D20934E0730934F0740935007509328
:1023A0005107B7D6C0925207D0925307E092540714
:1023B000F0925507C1010E94562CC1010E945A2C6F
:1023C000A8D604D6C1018CD7ABA1BCA11D921C928A
:1023D000EB85FC8511821082D8011D921C9240E091
:1023E00050E0B301C101EDD6EB85FC854081518100
:1023F000B201C101E6D6D8014D915C91B401C10191
:10240000E0D6C1010E945E2CBF85BB2309F44DC1FB
:1024100080D621E0FC01248748C1AA24A394B12CD2
:1024200096CCAA24A394B12CD9CCAA24A394B12CE1
:102430001CCD69E273E081010E521E4FC8010E945B
:1024400028276CE973E0C8010E94282768EB75E033
:10245000C8010E94282722E0A22EB12CE8CD65E217
:1024600073E081010E521E4FC8010E9428276CE9BB
:1024700073E0C8010E9428276DEC75E0C8010E9436
:10248000282792E0A92EB12C22CE61E273E08101CF
:102490000E521E4FC8010E9428276CE973E0C80144
:1024A0000E94282762EE75E0C8010E94282782E07A
:1024B000A82EB12C5CCE11821082F101E452FE4FA5
:1024C00080819181009749F46EE573E081010E529D
:1024D0001E4FC8010E942827C5C0019709F0D1C02E
:1024E00018D68C01FC0180819181A281B3811816DC
:1024F00019061A061B0644F081E090E0A0E0B0E067
:1025000080839183A283B383F80184819581A6811E
:10251000B781181619061A061B0644F081E090E0F0
:10252000A0E0B0E084839583A683B783F80180851B
:102530009185A285B385181619061A061B0644F064
:1025400081E090E0A0E0B0E080879187A287B38728
:102550006EE973E0CE0101960E94662763E275E0A2
:10256000CE0101960E9428276AEA74E0CE01019606
:102570000E94282760914A0770914B0780914C0771
:1025800090914D070E94AE4C6B017C01D8016D917A
:102590007D918D919C910E94AE4C9B01AC01C70135
:1025A000B6010E949C4EAB01BC01CE0101960E9477
:1025B000F8266AEB74E0CE0101960E94282760910C
:1025C0004E0770914F0780915007909151070E94DC
:1025D000AE4C6B017C01F801648175818681978125
:1025E0000E94AE4C9B01AC01C701B6010E949C4EFB
:1025F000AB01BC01CE0101960E94F8266AEC74E0A2
:10260000CE0101960E9428276091520770915307CE
:1026100080915407909155070E94AE4C6B017C014C
:10262000D80118966D917D918D919C911B970E9478
:10263000AE4C9B01AC01C701B6010E949C4EAB01A0
:10264000BC01CE0101960E94F826BE016F5F7F4F4C
:1026500081010E521E4FC8010E94362789819A813E
:102660000E94964756D5BC01CE01019616D4BE01F4
:102670006F5F7F4FC8010E94362789819A810E942F
:102680009647F101E452FE4F80819181019682309C
:1026900091051CF49183808302C011821082F101A4
:1026A000E652FE4F118210825CCA85E395E00E94DB
:1026B000053BC5010E94783B8CE993E00E94053BF5
:1026C00028D5B0924507A0924407C501E6960FB6FB
:1026D000F894DEBF0FBECDBFDF91CF911F910F9158
:1026E000FF90EF90DF90CF90BF90AF909F908F9032
:1026F0007F906F905F904F903F902F90089566234A
:1027000019F08DEA93E002C086EA93E00C94053B51
:102710000C9496470C9496478F929F92AF92BF92DB
:10272000CF92DF92EF92FF920F931F93CF93DF939D
:10273000EC018AE190E09E8B8D8B8BE190E0988F8D
:102740008F8B89E190E09A8F898F8FE090E09C8F4A
:102750008B8F8EE190E09E8F8D8F8EE090E098A31E
:102760008F8F85E490E09AA389A384E490E09CA3F2
:102770008BA3FE01E657FF4F80E290E096838583AE
:1027800081E290E0908787838FE190E09287818754
:102790001486138616861586108A178683E490E0C1
:1027A000928B818B82E490E0948B838BE658FF4F71
:1027B00083E290E09683858384E290E0908787832C
:1027C00082E290E0928781871486138616861586AA
:1027D000108A178681E490E0928B818B80E490E0F0
:1027E000948B838BE152FF4F1182108232961182BB
:1027F0001082329611821082CE010E94271DCE01D6
:102800004BD76E0182E8C81A8EEFD80A88248394C9
:10281000912CF601938E828E7E01F6E6EF1AFEEF82
:10282000FF0A84E090E0F701938F828F8E010A54B3
:102830001E4F88E090E0F801938F828F80E190E056
:10284000F6019183808381E190E095838483AA24BB
:10285000AA94BA2CB382A282B782A682C6010E9431
:102860004D35F601828580878385818787E190E0F9
:10287000F7019183808388E190E095838483B3821C
:10288000A282B782A682C7010E944D35F7018285D8
:102890008087838581878DE190E0F8019183808333
:1028A0008CE190E095838483B382A282B782A68272
:1028B000C8010E944D35F801828580878385818714
:1028C000EE5FFE4F808191813C9720813181369768
:1028D00040815181F601578B468B358B248B0197B4
:1028E00019F4B18EA08E03C0F601918E808EFE0188
:1028F000E654FD4F808191813C972081318136974C
:1029000040815181F701578B468B358B248B019782
:1029100019F48FEF9FEF03C081E090E0F701918FF2
:10292000808FFE01E454FD4F808191813C9720818E
:102930003181C655DD4F48815981F801578B468B4F
:10294000358B248B019719F48FEF9FEF03C081E043
:1029500090E0F801918F808FDF91CF911F910F91BF
:10296000FF90EF90DF90CF90BF90AF909F908F90AF
:1029700008952F923F924F925F926F927F928F9223
:102980009F92AF92BF92CF92DF92EF92FF920F93FE
:102990001F93CF93DF93CDB7DEB7CA57D1090FB6D8
:1029A000F894DEBF0FBECDBF8C01FC0110821182F6
:1029B0001282138214821582168217821086118663
:1029C0001286138614861586168617862C01F0E16A
:1029D0004F0E511CC2010E948A3268018AE8C80E5B
:1029E000D11CC6010E948A327801ECEFEE1AEEEF9C
:1029F000FE0AC7010E948A323801F2E86F1AFEEF20
:102A00007F0AC3010E94D335480186E6881A8EEFFB
:102A1000980AC4010E94D3355801EAE4AE1AEEEFD9
:102A2000BE0AC5010E94D3356EE973E0C8018E521B
:102A30009E4F0E946627F801E852FE4F11821082D5
:102A40003296118210823296118210823296118251
:102A50001082329610823196108231961082319611
:102A60001182108232961182108232961182108267
:102A700032961082319610823196108231961082F1
:102A80001182128213823496108211821282138272
:102A9000349610821182128213823496108211822F
:102AA000128213823496108211821282138234961B
:102AB0001082118212821382349610821182128245
:102AC00013823496108211821282138234961082FD
:102AD0001182128213823496108211821282138222
:102AE00034961082118212821382349610821182DF
:102AF00012821382349610821182128213823496CB
:102B000010821182128213823496108211821282F4
:102B1000138234961082319610823196108231964B
:102B200010821182128213823496108211821282D4
:102B3000138234961082118212821382349610828C
:102B40003196108231961082319610823196108221
:102B50003196108231961082319610823196108211
:102B60003196108231961082319610823196108201
:102B700031961082319610823196108231961082F1
:102B800031961082319610823196108231961082E1
:102B900031961082319610823196108231961082D1
:102BA0001182128213823496108211821282138251
:102BB00034961082118212821382D801A55ABD4F19
:102BC0008CE0E9E3F3E001900D928A95E1F7F801DA
:102BD000E959FD4F108211821282138234961082BD
:102BE0001182128213823496108211821282138211
:102BF000349611821082329611821082329611829E
:102C000010823296108211821282138234961082C0
:102C100011821282138234961082118212821382E0
:102C2000349610821182128213823496108211829D
:102C30001282138234961082118212821382349689
:102C40001182108232961182108232961182108285
:102C5000329610821182128213823496108211826F
:102C60001282138234961082118212821382349659
:102C70001082319610823196108231961182108224
:102C8000329611821082329611821082329611820F
:102C90001082329611821082329611821082329600
:102CA0001182108232961182108232961182108225
:102CB00032961182108232961182108232961182DF
:102CC000108232961182108232961182108218017F
:102CD000FEE32F1AFDEF3F0AF1011082CE010196AB
:102CE0000E948A328AE7FE013196D20101900D924C
:102CF0008A95E1F7CE0101960E948A328AE7FE01A9
:102D00003196D60101900D928A95E1F7CE01019698
:102D10000E948A328AE7FE013196D70101900D9216
:102D20008A95E1F788E5F801808B89E5F6018083D3
:102D30008AE5F7018083CE0101960E94D3358CE1AC
:102D4000FE013196D30101900D928A95E1F7CE01F3
:102D500001960E94D3358CE1FE013196D401019099
:102D60000D928A95E1F7CE0101960E94D3358CE150
:102D7000FE013196D50101900D928A95E1F7C801C7
:102D8000CBDCF1011082C658DF4F0FB6F894DEBFDE
:102D90000FBECDBFDF91CF911F910F91FF90EF90AC
:102DA000DF90CF90BF90AF909F908F907F906F906B
:102DB0005F904F903F902F900895CF93DF93809135
:102DC000930B9091940B892B51F483EC92E00E9429
:102DD0000147EC01CEDDD093940BC093930B80910F
:102DE000930B9091940BDF91CF9108954F925F9246
:102DF0006F927F928F929F92AF92BF92CF92DF920B
:102E0000EF92FF920F931F93CF93DF9300D01F9207
:102E1000CDB7DEB7FB011689078982889388A6841F
:102E2000B784C284D384E484F58446805780608468
:102E30007184428153816481758149835A836B8394
:102E40007C83BBDF1F921F921F920F931F939301EE
:102E5000820149815A816B817C810E941A0B0F90FB
:102E60000F900F900F900F9080E090E00F900F90D8
:102E70000F900F90DF91CF911F910F91FF90EF90E6
:102E8000DF90CF90BF90AF909F908F907F906F908A
:102E90005F904F90089508950895EF92FF920F93D9
:102EA0001F93CF93DF93CDB7DEB72E970FB6F8946D
:102EB000DEBF0FBECDBF8C016EE973E00E946627B6
:102EC00067EF75E0C8010E9428276091460770915E
:102ED000470780914807909149072AE0AE014F5F6C
:102EE0005F4F7A010E946548F70101900020E9F7E1
:102EF0003197AF014E195F09B701C8010E94CB2677
:102F00006CE973E0C8010E942827C8012E960FB60D
:102F1000F894DEBF0FBECDBFDF91CF911F910F910F
:102F2000FF90EF90089587EF95E00E94053B609138
:102F300046077091470780914807909149070E9482
:102F4000513B8CE993E00C94053B0F931F93CF9377
:102F5000DF93EC018AEF95E00E94053B8EEF95E050
:102F60000E94053B0DE81BE0F8016081CE01C7DB44
:102F700082E096E00E94053BF8016181CE01BFDB53
:102F800086E096E00E94053BF8016281CE01B7DB46
:102F90008AE096E00E94053BF8016381CE01AFDB39
:102FA0008EE096E00E94053BF8016481CE01A7DB2C
:102FB00082E196E00E94053BF8016581CE019FDB2E
:102FC000CE01DF91CF911F910F91ADCFCF92DF92C4
:102FD000EF92FF92CF93DF93EC0188819981AA81D0
:102FE000BB81181619061A061B0644F081E090E012
:102FF000A0E0B0E088839983AA83BB838C819D8104
:10300000AE81BF81181619061A061B0644F081E02E
:1030100090E0A0E0B0E08C839D83AE83BF83888581
:103020009985AA85BB85181619061A061B0644F051
:1030300081E090E0A0E0B0E088879987AA87BB870D
:1030400083E295E00E94053B8AEA94E00E94053BFA
:1030500060914A0770914B0780914C0790914D0702
:103060000E94AE4C6B017C01688179818A819B81D1
:103070000E94AE4C9B01AC01C701B6010E949C4E60
:1030800042E00E947D3B8AEB94E00E94053B609108
:103090004E0770914F0780915007909151070E9401
:1030A000AE4C6B017C016C817D818E819F810E9481
:1030B000AE4C9B01AC01C701B6010E949C4E42E0A0
:1030C0000E947D3B8AEC94E00E94053B6091520790
:1030D0007091530780915407909155070E94AE4C10
:1030E0006B017C01688579858A859B850E94AE4C41
:1030F0009B01AC01C701B6010E949C4E42E00E94B8
:103100007D3BCE01DF91CF91FF90EF90DF90CF908C
:103110000ACF80918B0B90918C0B892B91F58DE0D0
:1031200090E00E940147FC01148610924A07109219
:103130004B0710924C0710924D0710924E071092B9
:103140004F07109250071092510710925207109299
:103150005307109254071092550710928A0B109241
:10316000890B109246071092470710924807109259
:103170004907109245071092440790938C0B809357
:103180008B0B80918B0B90918C0B08950F931F9359
:10319000CF93DF938B01EA0181E593E00E94053B29
:1031A0008EE496E00E94053BF80180810E94463B38
:1031B000CE010E94783BADDFDF91CF911F910F913F
:1031C000B2CECF92DF92EF92FF920F931F93CF93E5
:1031D000DF93CDB7DEB728970FB6F894DEBF0FBEEA
:1031E000CDBF8B016A018E529E4F7C016DE473E06E
:1031F0000E9428276EE476E0C7010E942827F80184
:10320000808189831A8241E050E08E010F5F1F4F59
:10321000B801C7010E94CB264AE0B801C6010E944E
:103220005B48F80101900020E9F73197AF01401B9E
:10323000510BB801C7010E94CB266BDFBC01C8014E
:103240002CDEB801C7010E94362789819A810E942D
:10325000964728960FB6F894DEBF0FBECDBFDF911C
:10326000CF911F910F91FF90EF90DF90CF90089535
:10327000FC01DB01AD59BF4F8C91882319F022E08E
:1032800030E002C020E030E0DB01AB59BF4F8C9151
:10329000882311F023E030E0DB01AC59BF4F8C9163
:1032A000882311F024E030E0DB01AA59BF4F8C9154
:1032B000882311F026E030E0DA018D919C9182178D
:1032C000930721F091E0121613060CF090E0DA015A
:1032D0002D933C93992319F0A901CF0172CF089542
:1032E0008F929F92AF92BF92CF92DF92EF92FF9216
:1032F0000F931F93CF93DF93EC0189E493E00E9437
:10330000053B8AEA94E00E94053B6E0182E8C81AF8
:103310008EEFD80AC6010E94B3350E94AE4C4B0115
:103320005C01FE01E55AFD4F6081718182819381CC
:103330000E94AE4C9B01AC01C501B4010E949C4EA1
:1033400042E00E947D3B8AEB94E00E94053B7E01B7
:10335000E6E6EE1AEEEFFE0AC7010E94B3350E94C0
:10336000AE4C4B015C01FE01E15AFD4F6081718161
:10337000828193810E94AE4C9B01AC01C501B401D6
:103380000E949C4E42E00E947D3B8AEC94E00E94A9
:10339000053B8E010A541E4FC8010E94B3350E949E
:1033A000AE4C4B015C01CD59DD4F688179818A813A
:1033B0009B810E94AE4C9B01AC01C501B4010E94EF
:1033C0009C4E42E00E947D3BA4DEADDD85E493E0AF
:1033D0000E94053B8AEA94E00E94053BF601A08D1D
:1033E000B18D20893189428953890E94004E0E9403
:1033F000513B8AEB94E00E94053BF701A08DB18D13
:1034000020893189428953890E94004E0E94513B94
:103410008AEC94E00E94053BF801A08DB18D2089D3
:103420003189428953890E94004E0E94513B71DECE
:10343000DF91CF911F910F91FF90EF90DF90CF9090
:10344000BF90AF909F908F906ECD4F925F926F9292
:103450007F928F929F92AF92BF92CF92DF92EF9224
:10346000FF920F931F93CF93DF9300D01F92CDB79E
:10347000DEB70E941A0940903208509033086090DD
:103480003408709035080E941A0980903608909090
:103490003708A0903808B09039083BDEC0904A0742
:1034A000D0904B07E0904C07F0904D0732DEC701FB
:1034B000B6010E94AE4C6B017C01C301B2010E94B7
:1034C000AE4C9B01AC01C701B6010E949C4E2B0182
:1034D0003C0160914E0770914F0780915007909189
:1034E00051070E94AE4C6B017C01C501B4010E94E2
:1034F000AE4C9B01AC01C701B6010E949C4EAB01D2
:10350000BC0149835A836B837C8357DC1F921F92D3
:103510001F921F921F92812C912CA12CB12CC12C97
:10352000D12C760149815A816B817C818A019B0172
:10353000B301A2010E941A0B40DC1F921F921F923E
:103540001F921F9297018601B301A2010E941A0BDC
:1035500034DC1F921F921F921F921F9297018601C7
:10356000B701A6010E941A0B0FB6F894DEBF0FBE7A
:10357000CDBF80E090E00F900F900F900F90DF9103
:10358000CF911F910F91FF90EF90DF90CF90BF9060
:10359000AF909F908F907F906F905F904F90089525
:1035A000CF93DF9385E40E94D927EC01B2DD91E04F
:1035B000CD2B09F490E090938D0B84E40E94D927E1
:1035C000EC01A7DD91E0CD2B09F490E090938E0BF8
:1035D00083E40E94D927EC019CDD91E0CD2B09F416
:1035E00090E090938F0B82E40E94D927EC0191DD4B
:1035F00091E0CD2B09F490E09093900B81E40E9430
:10360000D927EC0186DD91E0CD2B09F490E0909371
:10361000910B80E40E94D927EC017BDD91E0CD2B5A
:1036200009F490E09093920BDF91CF910895CF939E
:10363000DF93EC012AEC30E04BEC50E069EC70E0F9
:103640000E944B2B2EEC30E04FEC50E06DEC70E024
:10365000CE010C960E944B2B24ED30E045ED50E05E
:1036600063ED70E0CE0148960E944B2B28ED30E0D0
:1036700049ED50E067ED70E0CE0184960E944B2B3F
:103680002EED30E04FED50E06DED70E0CE01C096D4
:10369000DF91CF910C944B2B2F923F924F925F92E0
:1036A0006F927F928F929F92AF92BF92CF92DF9252
:1036B000EF92FF920F931F93CF93DF93EC010E9441
:1036C0001A09FE01EF56FD4F8091120990911309DE
:1036D000918380830E941A09FE01ED56FD4F80916F
:1036E000160990911709918380830E941A09FE019F
:1036F000EB56FD4F80911A0990911B0991838083AD
:103700000E941A098E0109561D4F60913A09709165
:103710003B0980913C0990913D090E94AE4CF80113
:1037200060837183828393830E941A091E01F5E6E8
:103730002F1AFDEF3F0A60913E0970913F09809179
:103740004009909141090E94AE4CF1016083718360
:10375000828393830E941A0920E030E048EC52E40F
:10376000F80160817181828193810E949C4E2B01BE
:103770003C0120E030E048EC52E4F10160817181CD
:10378000828193810E949C4E4B015C0160914209B1
:103790007091430980914409909145090E94AE4C73
:1037A00020E030E048EC52E40E949C4E6B017C012A
:1037B0002AE037ED43E25CE3C301B2010E94354FDA
:1037C00018168CF420E030E046EC52E4C301B2015C
:1037D0000E94A84C87FD0FC0412C512C46EC642E52
:1037E00042E4742E08C05AE0452E57ED552E53E2A0
:1037F000652E5CE3752EF8014082518262827382ED
:103800002AE037ED43E25CE3C501B4010E94354F85
:1038100018168CF420E030E046EC52E4C501B40107
:103820000E94A84C87FD0FC0812C912C26ECA22E63
:1038300022E4B22E08C03AE0832E37ED932E33E215
:10384000A32E3CE3B32EF10180829182A282B38247
:103850002AE037ED43E25CE3C701B6010E94354F31
:1038600018168CF420E030E046EC52E4C701B601B3
:103870000E94A84C87FD0FC0C12CD12C86ECE82EED
:1038800082E4F82E08C09AE0C92E97EDD92E93E273
:10389000E92E9CE3F92EFE01E156FD4FC082D18254
:1038A000E282F3820E941A098091FA089091FB0843
:1038B000FE01EA55FD4F918380830E941A09809191
:1038C000FE089091FF08FE01E855FD4F918380832B
:1038D0000E941A098091020990910309FE01E655A0
:1038E000FD4F918380830E941A0980912209909153
:1038F0002309FE01E455FD4F918380830E941A093C
:103900008091260990912709FE01E255FD4F918390
:1039100080830E941A0980912A0990912B09FE0147
:10392000E055FD4F918380830E941A0980914A09D6
:1039300090914B09FE01EE54FD4F918380830E94CC
:103940001A0980914E0990914F09FE01EC54FD4FE8
:10395000918380830E941A098091520990915309A2
:10396000FE01EA54FD4F918380830E941A098091E1
:10397000620990916309FE01E854FD4F91838083B1
:103980000E941A098091660990916709FE01E65428
:10399000FD4F918380830E941A0980916A0990915A
:1039A0006B09FE01E454FD4F918380830E941A0944
:1039B0008091EA089091EB08A091EC08B091ED0895
:1039C000FE01ED55FD4F0197A105B10519F481E008
:1039D000808301C010820E941A098091EE089091A4
:1039E000EF08A091F008B091F108FE01EC55FD4FF1
:1039F0000197A105B10519F481E0808301C010820F
:103A00000E941A098091F2089091F308A091F4089D
:103A1000B091F508CB55DD4F0197A105B10519F41B
:103A200081E0888301C01882DF91CF911F910F91AF
:103A3000FF90EF90DF90CF90BF90AF909F908F90CE
:103A40007F906F905F904F903F902F9008952F92AE
:103A50003F924F925F926F927F928F929F92AF921E
:103A6000BF92CF92DF92EF92FF920F931F93CF936B
:103A7000DF93CDB7DEB760970FB6F894DEBF0FBE09
:103A8000CDBF988B8F870E941A09EF85F889E7517F
:103A9000FE4F81E040912208509123086091240854
:103AA00070912508452B462B472B09F480E0808335
:103AB0000E941A09EF85F889E651FE4F81E0409196
:103AC0002608509127086091280870912908452BF5
:103AD000462B472B09F480E080830E941A09EF856A
:103AE000F889E551FE4F81E040912A0850912B085A
:103AF00060912C0870912D08452B462B472B09F41B
:103B000080E080830E941A09809172089091730866
:103B1000A0917408B0917508EF85F889E451FE4FC3
:103B200080839183A283B3830E941A0980917608CF
:103B300090917708A0917808B0917908EF85F8897D
:103B4000E051FE4F80839183A283B3830E941A09C0
:103B500080917A0890917B08A0917C08B0917D08B3
:103B6000EF85F889EC50FE4F80839183A283B38365
:103B70000E941A0980914A0890914B08A0914C0824
:103B8000B0914D08EF85F889EC5FFD4F80839183FC
:103B9000A283B3830E941A0980914E0890914F0826
:103BA000A0915008B0915108EF85F889E85FFD4F6A
:103BB00080839183A283B3830E941A098091520863
:103BC00090915308A0915408B0915508EF85F88959
:103BD000E45FFD4F80839183A283B3830E941A091F
:103BE00080915A0890915B08A0915C08B0915D08A3
:103BF000EF85F889E05FFD4F80839183A283B383D3
:103C00000E941A0980915E0890915F08A091600857
:103C1000B0916108EF85F889EC5EFD4F8083918358
:103C2000A283B3830E941A0980916208909163086D
:103C3000A0916408B0916508EF85F889E85EFD4FB2
:103C400080839183A283B3830E941A098091FA072B
:103C50009091FB07A091FC07B091FD07EF85F889D3
:103C6000E45EFD4F80839183A283B3830E941A098F
:103C70008091FE079091FF07A0910008B091010884
:103C8000EF85F889E05EFD4F80839183A283B38343
:103C90000E941A098091020890910308A0910408DB
:103CA000B0910508EF85F889EC5DFD4F8083918325
:103CB000A283B3830E941A09EF85F889E85DFD4F5E
:103CC00081E02091D2073091D3072130310509F0EE
:103CD00080E080830E941A09EF85F889E75DFD4F37
:103CE00081E02091D6073091D7072130310509F0C6
:103CF00080E080830E941A09EF85F889E65DFD4F18
:103D000081E02091DA073091DB072130310509F09D
:103D100080E080830E941A09EF85F889EA5BFD4FF5
:103D200081E04091AA075091AB076091AC07709178
:103D3000AD07452B462B472B09F480E080830E947A
:103D40001A09EF85F889E95BFD4F81E04091AE07E4
:103D50005091AF076091B0077091B107452B462B8A
:103D6000472B09F480E080830E941A09EF85F889C7
:103D7000E85BFD4F81E04091B2075091B30760913D
:103D8000B4077091B507452B462B472B09F480E00B
:103D900080830E941A09EF85F889E75BFD4F81E077
:103DA0004091820850918308609184087091850841
:103DB000452B462B472B09F480E080830E941A098B
:103DC000EF85F889E65BFD4F81E0409186085091D0
:103DD00087086091880870918908452B462B472BEE
:103DE00009F480E080830E941A09EF85F889E55B79
:103DF000FD4F81E040918A0850918B0860918C08BA
:103E000070918D08452B462B472B09F480E0808369
:103E10000E941A09EF85F889E45BFD4F81E020914B
:103E2000BA073091BB072130310509F080E080836B
:103E30000E941A09EF85F889E35BFD4F81E020912C
:103E4000BE073091BF072130310509F080E0808343
:103E50000E941A09EF85F889E25BFD4F81E020910D
:103E6000C2073091C3072130310509F080E080831B
:103E70000E941A098091820790918307A09184077C
:103E8000B0918507EF85F889E15BFD4F80839183D1
:103E9000A283B3830E941A098091860790918707B5
:103EA000A0918807B0918907EF85F889ED5AFD4FF9
:103EB00080839183A283B3830E941A0980918A0729
:103EC00090918B07A0918C07B0918D07EF85F889B1
:103ED000E95AFD4F80839183A283B3830E941A091C
:103EE000EF85F889E65CFD4F81E0409192075091A3
:103EF00093076091940770919507452B462B472BAC
:103F000009F480E080830E941A09EF85F889E55C56
:103F1000FD4F81E040919607509197076091980777
:103F200070919907452B462B472B09F480E080833D
:103F30000E941A09EF85F889E45CFD4F81E0409109
:103F40009A0750919B0760919C0770919D07452BA4
:103F5000462B472B09F480E080830E941A09809148
:103F60008A0990918B09A0918C09B0918D09EF85F8
:103F7000F889E55DFD4F80839183A283B3830E941E
:103F80001A0980918E0990918F09A0919009B091A2
:103F90009109EF85F889E15DFD4F80839183A283CC
:103FA000B3830E941A098091920990919309A0917C
:103FB0009409B0919509EF85F889ED5CFD4F8083F8
:103FC0009183A283B3830E941A09EF85F889E35C89
:103FD000FD4F81E02091EA073091EB072130310558
:103FE00009F080E08083EF85F889E25CFD4F108264
:103FF000EF85F889E15CFD4F10820E941A09EF8578
:10400000F889E05CFD4F81E02091E6073091E707F9
:104010002130310509F080E08083EF85F889EF5B7E
:10402000FD4F1082EF85F889EE5BFD4F10820E94F4
:104030001A09EF85F889ED5BFD4F81E020910A08B0
:1040400030910B082130310509F080E080830E9417
:104050001A09EF85F889EC5BFD4F81E020910E088D
:1040600030910F082130310509F080E080830E94F3
:104070001A09EF85F889EB5BFD4F81E0209112086A
:10408000309113082130310509F080E080830E94CF
:104090001A09EF85F889E95CFD4F81E020919A09C2
:1040A00030919B092130310509F080E080830E9426
:1040B0001A09EF85F889E85CFD4F81E020919E099F
:1040C00030919F092130310509F080E080830E9402
:1040D0001A09EF85F889E75CFD4F81E02091A2097C
:1040E0003091A3092130310509F080E080830E94DE
:1040F0001A090F851889055A1D4F80913208909131
:104100003308A0913408B0913508F8018083918379
:10411000A283B3830E941A09EF84F888F1EAEF1AA8
:10412000FDEFFF0A8091360890913708A09138087A
:10413000B0913908F70180839183A283B3830E94F1
:104140001A0980913A0890913B08A0913C08B091DF
:104150003D082F8538892D593D4FF9018083918382
:10416000A283B383F8014081518162817381141667
:1041700015061606170644F041E050E060E070E0D6
:104180004083518362837383F7014081518162814F
:104190007381141615061606170644F041E050E028
:1041A00060E070E0408351836283738318161906C0
:1041B0001A061B064CF081E090E0A0E0B0E0F901A7
:1041C00080839183A283B383D9018D909D90AD901C
:1041D000BC90F701C080D180E280F380D8014D907F
:1041E0005D906D907C900E948918FC014082518204
:1041F00062827382C482D582E682F782808691864B
:10420000A286B386EF85F889E95CFD4FB081B9835A
:10421000EF85F889E55DFD4F80819181A281B381B1
:104220004F8558894D5B5D4FFA01F081FB834F85C7
:104230005889445B5D4FFA01F081FA834F855889B4
:10424000435C5D4FFA01F081FF834F855889405CE4
:104250005D4FFA01F081F8874F855889475B5D4FC4
:10426000FA01F081F9874F8558894A5B5D4FFA0161
:10427000F081FA87EF85F889E85DFD4F2080EF85B2
:10428000F889E751FE4F3080EF85F889E15BFD4FFB
:104290004081518162817381EF85F889E45EFD4F31
:1042A0000081118122813381EF85F889E05FFD4F24
:1042B000C080D180E280F380EF85F889EC5FFD4F0C
:1042C00080809180A280B380EF85F889E451FE4F11
:1042D0004080518062807380EF85F88940A651A6A6
:1042E00062A673A684A695A6A6A6B7A6C0AAD1AABA
:1042F000E2AAF3AA04AB15AB26AB37AB40AF51AF84
:1043000062AF73AF34AE25AE2A8525A3398536A3B7
:104310004A8147A340E450E060E070E0E05CFF4F7A
:1043200040835183628373832885EF85F88926AFA4
:104330003F8137AFAF014C5B5F4F2B81FA01208388
:10434000EF85F889EB5BFF4F80839183A283B38372
:10435000EF85F889E75BFF4F39813083AF85B889F6
:1043600055968D919C9156978633910589F481EAF3
:104370009CE2FD01E658FF4F9183808332961182C3
:1043800010828FE99CE2369691838083329630C00A
:104390008C33910589F489E99CE2EF85F889E65828
:1043A000FF4F91838083EF85F889E458FF4F118296
:1043B000108287E99CE212C08E97E1F481E99CE2C9
:1043C000EF85F889E658FF4F91838083EF85F88960
:1043D000E458FF4F118210828BE89CE2EF85F88948
:1043E000EE57FF4F91838083EF85F889EC57FF4F9D
:1043F00011821082EF85F889838D948D4A97D1F4CC
:104400008DE99CE2E258FF4F91838083EF85F88924
:10441000E058FF4F118210828BE99CE2EF85F8890A
:10442000EA57FF4F91838083EF85F889E857FF4F64
:1044300011821082EF85F889E85CFD4F2081298385
:10444000EF85F889E15DFD4F408051806280738087
:10445000EF85F889EC5BFD4F30813B83EF85F88970
:10446000E35BFD4F9081EF85F889E25CFD4F408171
:104470004F83EF85F889EF5BFD4F50815887EF85BB
:10448000F889E65BFD4F8081EF85F889E95BFD4F98
:10449000A081AA87EF85F889E75DFD4F2080EF8531
:1044A000F889E651FE4F3080EF85F889ED5AFD4FCF
:1044B00020813181428153812B873C874D875E87E4
:1044C000EF85F889E05EFD4F408151816281738103
:1044D000EF85F889EC5EFD4FC080D180E280F380EB
:1044E000EF85F889E85FFD4F80809180A280B380DE
:1044F000EF85F889E657FF4F2F85388920513E4FC9
:10450000D9010D911D912D913C91008F118F228F1A
:10451000338F848E958EA68EB78EC0A2D1A2E2A2D2
:10452000F3A244A355A366A377A32B853C854D85B1
:104530005E8520A731A742A753A734A625A63A85B2
:10454000358B868B978B80E490E0A0E0B0E080AB69
:1045500091ABA2ABB3AB488546A75F8157A78B81D0
:1045600084AB45AA56AA67AA70AE998191AF85819E
:1045700096818633910589F481EA9CE2AF85B889FA
:10458000AC50BF4F8D939C93AF85B889AA50BF4F55
:104590001D921C928FE99CE226C08C33910589F410
:1045A00089E99CE2AF85B889AC50BF4F8D939C934D
:1045B000AF85B889AA50BF4F1D921C9287E99CE233
:1045C00012C08E97E1F481E99CE2AF85B889AC50C6
:1045D000BF4F8D939C93AF85B889AA50BF4F1D9252
:1045E0001C928BE89CE2AF85B889A450BF4F8D9395
:1045F0009C93AF85B889A250BF4F1D921C928385B2
:1046000094854A97D9F48DE99CE2EF85F889E850C2
:10461000FF4F91838083EF85F889E650FF4F118229
:1046200010828BE99CE2EF85F889F3959183808372
:10463000EF85F889EE5FFE4F11821082EF85F889D1
:10464000E75CFD4FA081A9832F8538892D5C3D4F04
:10465000D9018D919D910D90BC91A02D8B839C8350
:10466000AD83BE83EF85F889EB5BFD4FB081BA83E4
:10467000EF85F889E25BFD4F20812F83EF85F88974
:10468000E15CFD4F30813887EF85F889EE5BFD4FA7
:1046900040814987EF85F889E55BFD4F2080EF85F4
:1046A000F889E85BFD4F3080EF85F889E65DFD4FC6
:1046B0003081EF85F889E551FE4F2081EF85F8893B
:1046C000E95AFD4F80819181A281B381EF85F889FC
:1046D000EC5DFD4F4081518162817381EF85F889E6
:1046E000E85EFD4FC080D180E280F380EF85F889DD
:1046F000E45FFD4F80809180A280B3800F85188990
:104700000C5F1E4FEF85F889EC50FE4F40805180C2
:1047100062807380F801408E518E628E738E848E1B
:10472000958EA68EB78EC0A2D1A2E2A2F3A244A318
:1047300055A366A377A380A791A7A2A7B3A724A791
:1047400035A7358A268A2F81278B80E490E0A0E068
:10475000B0E080AB91ABA2ABB3AB298526A738857F
:1047600037A74A8144AB8B819C81AD81BE8185ABEB
:1047700096ABA7ABB0AF298121AF858196818633F7
:10478000910589F481EA9CE2EF85F889E259FE4FB0
:1047900091838083EF85F889E059FE4F1182108262
:1047A0008FE99CE226C08C33910589F489E99CE26B
:1047B000EF85F889E259FE4F91838083EF85F88970
:1047C000E059FE4F1182108287E99CE212C08E9759
:1047D000E1F481E99CE2EF85F889E259FE4F91838B
:1047E0008083EF85F889E059FE4F118210828BE8B3
:1047F0009CE2EF85F889EA58FE4F91838083EF852C
:10480000F889E858FE4F11821082D8011B968D91CD
:104810009C911C974A97E1F48DE99CE2EF85F88919
:10482000EE58FE4F91838083EF85F889EC58FE4F58
:10483000118210828BE99CE2EF85F889E658FE4FE1
:1048400091838083EF85F889E458FE4F11821082AE
:10485000EF85F889E65CFD4F20818F859889409629
:10486000222319F00E94072E02C00E94F52DEF8529
:10487000F889E55CFD4F20818F85988986579F4F89
:10488000222319F00E94072E02C00E94F52DEF8509
:10489000F889E45CFD4F80818823D9F0C8016096D7
:1048A0000FB6F894DEBF0FBECDBFDF91CF911F9141
:1048B0000F91FF90EF90DF90CF90BF90AF909F90BF
:1048C0008F907F906F905F904F903F902F900C94BF
:1048D000072EC80160960FB6F894DEBF0FBECDBF9D
:1048E000DF91CF911F910F91FF90EF90DF90CF90CC
:1048F000BF90AF909F908F907F906F905F904F9000
:104900003F902F900C94F52DCF92DF92EF92FF9273
:104910000F931F93CF93DF936C017A018B01C0E05B
:10492000D0E0CE15DF0589F0D8016D918D01D6015B
:10493000ED91FC910190F081E02DC6011995892B34
:1049400011F47E0102C02196ECCFC701DF91CF9117
:104950001F910F91FF90EF90DF90CF9008950895F1
:1049600080E090E00895FC01538D448D252F30E0C8
:10497000842F90E0821B930B541710F0CF9608956C
:1049800001970895FC01918D828D981761F0828DB9
:10499000DF01A80FB11D5D968C91928D9F5F9F7373
:1049A000928F90E008958FEF9FEF0895FC01918D15
:1049B000828D981731F0828DE80FF11D858D90E082
:1049C00008958FEF9FEF0895FC01918D228D892F1F
:1049D00090E0805C9F4F821B91098F739927089507
:1049E00088EA9BE0F1DF21E0892B09F420E0822FA7
:1049F0000895FC01848DDF01A80FB11DA35ABF4F9C
:104A00002C91848D90E001968F739927848FA689CD
:104A1000B7892C93A089B1898C9180648C93938DF4
:104A2000848D981306C00288F389E02D80818F7DE4
:104A300080830895EF92FF920F931F93CF93DF939C
:104A4000EC0181E0888F9B8D8C8D981305C0E889DF
:104A5000F989808185FD23C0F62E0B8D10E00F5F54
:104A60001F4F0F731127E02E8C8DE8120BC00FB66D
:104A700007FCFACFE889F989808185FFF5CFCE015F
:104A8000B8DFF2CF8B8DFE01E80FF11DE35AFF4F27
:104A9000F0820B8FEA89FB898081806207C0EE89F2
:104AA000FF896083E889F98980818064808381E05F
:104AB00090E0DF91CF911F910F91FF90EF900895BB
:104AC000CF93DF93EC01888D8823C1F0EA89FB89BD
:104AD000808185FD05C0A889B9898C9186FD0EC0AD
:104AE0000FB607FCF5CF808185FFF2CFA889B98981
:104AF0008C9185FFEDCFCE017CDFE8CFDF91CF91A8
:104B0000089580E090E0892B19F06ADF811125C0BB
:104B100080E090E0892B41F080E090E0892B21F04B
:104B20000E94000081111CC080E090E0892B41F0C0
:104B300080E090E0892B21F00E940000811113C0D9
:104B400080E090E0892BA1F080E090E0892B81F05B
:104B50000E94000081110AC008950E940000D8CF71
:104B60000E940000E1CF0E940000EACF0C940000F8
:104B7000089590E0FC013197E231F10508F04EC054
:104B80008827EC59FE4F8F4F0C943D4F8091800049
:104B90008F7703C0809180008F7D8093800008957F
:104BA00080918000877FF9CF84B58F7702C084B56C
:104BB0008F7D84BD08958091B0008F7703C0809170
:104BC000B0008F7D8093B0000895809190008F7722
:104BD00007C0809190008F7D03C080919000877FF7
:104BE0008093900008958091A0008F7707C08091F6
:104BF000A0008F7D03C08091A000877F8093A000DC
:104C00000895809120018F7707C0809120018F7DCA
:104C100003C080912001877F8093200108953FB7D2
:104C2000F89480919E0B90919F0BA091A00BB09156
:104C3000A10B26B5A89B05C02F3F19F00196A11D19
:104C4000B11D3FBFBA2FA92F982F8827820F911D22
:104C5000A11DB11DBC01CD0142E0660F771F881F69
:104C6000991F4A95D1F708950E942C500C949647AD
:104C70000C9496470F931F93CF93DF93EC01888199
:104C80009981009729F02A813B812617370788F4FC
:104C90008B016F5F7F4F0E94454F009761F09983B2
:104CA00088831B830A832C813D81232B11F4FC0113
:104CB000108281E001C080E0DF91CF911F910F91C0
:104CC00008958F929F92AF92BF92CF92DF92EF9210
:104CD000FF920F931F930E94DD1662E070E00E9426
:104CE000F335892BD1F40E94DD1621E02F931F921A
:104CF0001F921F921F92812C912CA12CB12CC12CA0
:104D0000D12C760197018601B701A6010E941A0BEA
:104D10000F900F900F900F900F9080E090E01F91F8
:104D20000F91FF90EF90DF90CF90BF90AF909F904A
:104D30008F9008958F929F92AF92BF92CF92DF9201
:104D4000EF92FF920F931F930E94DD161F9221E0B6
:104D50002F931F921F921F92812C912CA12CB12C6A
:104D6000C12CD12C760197018601B701A6010E94C2
:104D70001A0B0F900F900F900F900F9080E090E023
:104D80001F910F91FF90EF90DF90CF90BF90AF9069
:104D90009F908F900895EF92FF920F931F93CF9360
:104DA000DF93FC01248135816115710511F480E0E8
:104DB00018C041155105A1F07B01EC018A01020FD9
:104DC000131FB80157DF882391F3288139818C8123
:104DD0009D81B701820F931F0E9442501D830C8357
:104DE00081E0DF91CF911F910F91FF90EF90089597
:104DF000EF92FF920F931F93CF93DF93CDB7DEB760
:104E000064970FB6F894DEBF0FBECDBF7C01CB0117
:104E1000BA018E010F5F1F4F22E044E00E94E2467C
:104E2000BC01FC0101900020E9F73197AF01481B5C
:104E3000590BC701B0DF64960FB6F894DEBF0FBE02
:104E4000CDBFDF91CF911F910F91FF90EF9008950B
:104E50006115710549F0FB0101900020E9F73197D8
:104E6000AF01461B570B97CF80E00895FB014481AB
:104E70005581608171818FCFEF92FF920F931F93C5
:104E8000CF93DF93EC017B018A01BA01F3DE288125
:104E9000398181110DC02115310519F0C9010E9418
:104EA0009647198218821D821C821B821A8206C0B4
:104EB0001D830C83B701C9010E944250CE01DF91CE
:104EC000CF911F910F91FF90EF900895FC011182F7
:104ED000108213821282158214826115710549F0C5
:104EE000FB0101900020E9F73197AF01461B570BFA
:104EF000C3CF08951F920F920FB60F9211240BB6D5
:104F00000F922F933F934F935F936F937F938F9362
:104F10009F93AF93BF93EF93FF9388EA9BE069DD84
:104F2000FF91EF91BF91AF919F918F917F916F9181
:104F30005F914F913F912F910F900BBE0F900FBE3D
:104F40000F901F9018951F920F920FB60F92112479
:104F50000BB60F922F938F939F93EF93FF93E09154
:104F6000B80BF091B90B8081E091BE0BF091BF0BB3
:104F700082FD12C090818091C10B8F5F8F73209151
:104F8000C20B821751F0E091C10BF0E0E855F44FED
:104F9000958F8093C10B01C08081FF91EF919F910C
:104FA0008F912F910F900BBE0F900FBE0F901F90FF
:104FB0001895CF93DF93282F30E0F901EF5DFB4F79
:104FC0008491F901E550FB4FD491F901EB54FB4F6B
:104FD000C491CC2389F08111CCDDEC2FF0E0EE0FF1
:104FE000FF1FE556FB4FA591B491EC91ED2381E0B5
:104FF00090E021F480E002C080E090E0DF91CF916A
:1050000008951F93CF93DF93282F30E0F901EF5DD0
:10501000FB4F8491F901E550FB4FD491F901EB541A
:10502000FB4FC491CC23C1F0162F8111A2DDEC2FD0
:10503000F0E0EE0FFF1FEF57FB4FA591B4918FB734
:10504000F894111105C09C91ED2FE095E92302C061
:10505000EC91ED2BEC938FBFDF91CF911F910895D1
:10506000CF92DF92EF92FF920F931F93CF93DF9334
:105070006C018B017A01EC01CB56D44F888187FFFC
:1050800004C0FB011182108224C08CE08C9D900131
:105090008D9D300D11248881A901480F511D87FD78
:1050A0005A958091DD0C90E04817590794F4888157
:1050B000A901480F511D87FD5A95CA01FA01EE0F4B
:1050C000FF1F8E0F9F1FFC01E35BF34F808186FD66
:1050D00019C088818F5F88838CE08C9D90018D9DA5
:1050E000300D11248881A901480F511D87FD5A9563
:1050F0008091DD0C90E048175907B4F488818C301A
:105100003CF112C08881280F311D87FD3A95F901C5
:10511000EE0FFF1F2E0F3F1FF901E35BF34F80815E
:1051200060E08F736EDFD5CFF801808191810496A6
:1051300080349C4918F480E49CE904C0F801808123
:1051400091810496F701918380838FEF888344C017
:10515000F801408151818881B901680F711D87FD77
:105160007A95CB01FB01EE0FFF1F8E0F9F1FFC01F5
:10517000E35BF34F81819281840F951FF701918347
:1051800080838881A901480F511D87FD5A95CA0166
:10519000FA01EE0FFF1F8E0F9F1FFC01E35BF34F21
:1051A000808186FF19C08881280F311D87FD3A95BF
:1051B000F901EE0FFF1F2E0F3F1FF901E35BF34FC5
:1051C000808161E08F73DF91CF911F910F91FF90EC
:1051D000EF90DF90CF9015CFDF91CF911F910F917E
:1051E000FF90EF90DF90CF900895CF93DF9390E002
:1051F000FC01E550FB4F2491FC01EB54FB4F8491E3
:10520000882361F190E0880F991FFC01E959FB4F59
:10521000C591D491FC01EF57FB4FA591B491611159
:1052200009C09FB7F8948881209582238883EC91E8
:105230002E230BC0623061F49FB7F8943881822F1F
:10524000809583238883EC912E2B2C939FBF06C0DF
:105250008FB7F894E8812E2B28838FBFDF91CF91F1
:1052600008958230910538F0880F991F880F991F93
:1052700005970197F1F708958F929F92AF92BF9291
:10528000CF92DF92EF92FF926B017C01C8DC4B0161
:105290005C01C114D104E104F104E9F0C0DCDC01DB
:1052A000CB0188199909AA09BB09883E9340A10539
:1052B000B10578F321E0C21AD108E108F10888EEBF
:1052C000880E83E0981EA11CB11CC114D104E10416
:1052D000F10421F7DECFFF90EF90DF90CF90BF90E9
:1052E000AF909F908F9008952FB7F89460919A0B8C
:1052F00070919B0B80919C0B90919D0B2FBF0895FB
:105300001F920F920FB60F9211242F933F938F93FA
:105310009F93AF93BF9380919A0B90919B0BA09119
:105320009C0BB0919D0B3091990B23E0230F2D37EF
:1053300020F40196A11DB11D05C026E8230F029699
:10534000A11DB11D2093990B80939A0B90939B0BF9
:10535000A0939C0BB0939D0B80919E0B90919F0B03
:10536000A091A00BB091A10B0196A11DB11D80933E
:105370009E0B90939F0BA093A00BB093A10BBF919A
:10538000AF919F918F913F912F910F900FBE0F90F2
:105390001F901895CF92DF92EF92FF92CF93DF93F9
:1053A000EC01603282E078070CF03DC077FD06C06A
:1053B000653B71052CF064EB70E002C060E070E0CA
:1053C000898128E830E06901C81AD10887FDD394A3
:1053D000CC0CDD1CCC0CDD1C0D2C000CEE08FF08E9
:1053E0008A8128E532E0281B310987FD3395220F99
:1053F000331F220F331FC901330FAA0BBB0B9C01B4
:10540000AD012C193D094E095F09DB010E94004ED8
:1054100024EB30E040E050E00E94DA4DC20ED31E93
:10542000E41EF51EB6018881803380F5998148E835
:1054300050E0491B510997FD5395440F551F440FE8
:10544000551F6417750784F09A8128E532E0291BFF
:10545000310997FD3395220F331F220F331FAB0104
:10546000261737070CF4A90142505109440F551F64
:105470002FB7F89490E0FC01EE0FFF1F8E0F9F1FD7
:10548000FC01E35BF34F528341832FBFDF91CF9148
:10549000FF90EF90DF90CF9008951F920F920FB67C
:1054A0000F9211240BB60F922F933F934F935F935C
:1054B0006F937F938F939F93AF93BF93EF93FF93DC
:1054C00048E251E064E271E080E090E0C9DDFF91E4
:1054D000EF91BF91AF919F918F917F916F915F916C
:1054E0004F913F912F910F900BBE0F900FBE0F90D9
:1054F0001F9018951F920F920FB60F9211240BB6A2
:105500000F922F933F934F935F936F937F938F935C
:105510009F93AF93BF93EF93FF9348EA50E064EA01
:1055200070E083E090E09CDDFF91EF91BF91AF913F
:105530009F918F917F916F915F914F913F912F91AB
:105540000F900BBE0F900FBE0F901F9018951F92DB
:105550000F920FB60F9211240BB60F922F933F9319
:105560004F935F936F937F938F939F93AF93BF936B
:10557000EF93FF9348E950E064E970E082E090E047
:105580006FDDFF91EF91BF91AF919F918F917F91CF
:105590006F915F914F913F912F910F900BBE0F90A4
:1055A0000FBE0F901F9018951F920F920FB60F927B
:1055B00011240BB60F922F933F934F935F936F93EA
:1055C0007F938F939F93AF93BF93EF93FF9348E89D
:1055D00050E064E870E081E090E042DDFF91EF91FF
:1055E000BF91AF919F918F917F916F915F914F91FB
:1055F0003F912F910F900BBE0F900FBE0F901F90F9
:10560000189508950F931F93CF93DF93FC0120818A
:10561000318121153105D1F1EC01822FCADC21E065
:10562000892B09F420E02B876A85261729F01E8232
:105630001F82188619860BC08E819F81A885B98527
:105640000196A11DB11D8E839F83A887B9870E8106
:105650001F81288539858A819B81AC81BD8108178E
:1056600019072A073B0794F081E068278881C9DC85
:105670000990D881C02D0E94A53440E050E0BE01C1
:10568000DF91CF911F910F910C949B09DF91CF91E6
:105690001F910F910895CF92DF92EF92FF920F9397
:1056A0001F93CF93DF937C016B018A01E9010E9474
:1056B0001A09F601EE0FFF1FEE0FFF1FEA5AF84F0F
:1056C00080819181F701918380830E941A09000FE4
:1056D000111F000F111FF801EA5AF84F81E04081B5
:1056E000518162817381413051056105710509F075
:1056F00080E0F70182870E941A09CC0FDD1FCC0FD2
:10570000DD1FCA5AD84F88819981AA81BB81F701D0
:1057100082839383A483B5831682178210861186B1
:10572000DF91CF911F910F91FF90EF90DF90CF907D
:10573000089508952F923F924F925F926F927F92B9
:105740008F929F92AF92BF92CF92DF92EF92FF9291
:105750000F931F93CF93DF9300D000D0CDB7DEB768
:105760009E838D834B015A013A8329831801FC8261
:10577000EB82FA01408051806280738020E030E04B
:10578000A901C301B2010E94354F181674F4F60145
:105790002081318142815381C301B2010E94374E81
:1057A000F5016083718382839383ED81FE81E05AEA
:1057B000FF4F8081F401008D118DC088D188E2886F
:1057C000F388F1014080518062807380D801A70185
:1057D0009601882341F00E94004E641575058605E8
:1057E000970544F023C00E94004E461657066806EF
:1057F0007906E4F4F501408051806280738020E0F6
:1058000030E04AEF56E4C301B2010E94A84C87FF82
:105810000DC020E030E040E85FE3C301B2010E9428
:10582000384EF5016083718382839383D801A70189
:1058300096010E94004EF1016083718382839383FD
:105840000D811E81025C1F4FF80180819181A28130
:10585000B381E981FA8180839183A283B383EB8151
:10586000FC8180819181892B41F0C4010E94B33574
:10587000F801608371838283938326960FB6F89430
:10588000DEBF0FBECDBFDF91CF911F910F91FF9073
:10589000EF90DF90CF90BF90AF909F908F907F90D0
:1058A0006F905F904F903F902F9008950E948918BD
:1058B0000C94D01A0E9489180C94A517CF93DF93EB
:1058C000EC01FC01EE53FD4F1082E858F109808194
:1058D000811103C0CE01409688D1FE01E55CFD4FE9
:1058E0008081811104C0CE0186579F4F7ED1FE0179
:1058F000E45CFD4F8081811104C0CE018C5F9E4F1E
:1059000074D164E670E080E090E0DF91CF91B4CC98
:105910008FEF9FEF0895EBE0F1E08081877F808338
:105920000895EBE0F1E080818860808308958E988F
:1059300008958E9A089514980895149A0895889851
:105940000895889A08950C9496470C9496470C9461
:1059500096470C9496470C9496470F931F93CF93BA
:10596000DF93FB01C2A1D3A1068D178D8091A20BFD
:105970009091A30B892B41F481E090E00E940147B4
:105980009093A30B8093A20B0430110539F00530DE
:10599000110541F4BE0181EE9CE003C0BE018EED15
:1059A0009CE0F8DC80E090E0DF91CF911F910F91B7
:1059B00008958F929F92AF92BF92CF92DF92EF9213
:1059C000FF920F931F930E94DD161F921F9221E0FA
:1059D0002F931F921F92812C912CA12CB12CC12CA2
:1059E000D12C760197018601B701A6010E941A0BFE
:1059F0000F900F900F900F900F9080E090E01F910C
:105A00000F91FF90EF90DF90CF90BF90AF909F905D
:105A10008F9008950E9489180E94E61780E090E018
:105A2000089560E0FC018385ECCA60E0FC0185819B
:105A3000E8CA61E0FC018385E4CA61E0FC0185817C
:105A4000E0CACF93DF93FB01C68DD78D0E941A0960
:105A5000BE010E94D70880E090E0DF91CF910895C9
:105A6000CF93DF938091A40B9091A50B892BF1F438
:105A70008CE390E00E940147EC01FC01CC9611827E
:105A800010823C96E817F907D1F7198218821D8613
:105A90001C86198E188E1DA21CA219AA18AACE0146
:105AA0000E94171BD093A50BC093A40B8091A40B4D
:105AB0009091A50BDF91CF910895089508950895D1
:105AC00008951F920F920FB60F9211240BB60F92EA
:105AD0002F933F934F935F936F937F938F939F93F6
:105AE000AF93BF93EF93FF93E0914207F091430789
:105AF0001995FF91EF91BF91AF919F918F917F91F8
:105B00006F915F914F913F912F910F900BBE0F902E
:105B10000FBE0F901F901895CF93DF93EC01FC01FF
:105B2000E759FF4F1082379781E0808360E08D81D5
:105B300068DA8F859889892B29F060E08B85DF9161
:105B4000CF915FCADF91CF910895CF93DF93EC019E
:105B50008B892FDA2E8930E08217930711F48F8911
:105B600001C080E0DF91CF910895CF93DF93EC01E6
:105B700089891FDA2E8930E08217930711F48F8903
:105B800001C080E0DF91CF910895CF93DF93EC01C6
:105B90008DA5882311F061E001C060E08F8131DACA
:105BA0008EA5882329F08FA5882311F061E001C01C
:105BB00060E08D85DF91CF9124CACF93DF93EC0114
:105BC0008DA5882311F060E001C061E08F8119DAB2
:105BD0008EA5882329F08FA5882311F060E001C0ED
:105BE00061E08D85DF91CF910CCACF93DF93EC01FB
:105BF00061E0898506DA8EA5882319F061E08F853A
:105C000000DAC959DF4F1882DF91CF910895CF9301
:105C1000DF93EC0160E08985F4D98EA5882319F023
:105C200060E08F85EED9C959DF4F81E08883DF912D
:105C3000CF910895CF92DF92EF92FF920F931F932F
:105C4000CF93DF93FC0142AF53AF64AF75AFDC017C
:105C5000DE964D935D936D937C93139714960D93FD
:105C60001D932D933C931397EC01CA5BDF4FE882A1
:105C700084A9882389F084A5811109C037FF0CC04D
:105C80001D921D921D921C92139781E006C0101662
:105C9000110612061306A4F380E045A956A967A9C8
:105CA00070AD14161506160617063CF591AD99232E
:105CB00021F10D911D912D913C911397680179016E
:105CC00037FF07C0CC24DD247601C01AD10AE20ACE
:105CD000F30A4C155D056E057F057CF437FF07C0A0
:105CE00070956095509541955F4F6F4F7F4F4D93E5
:105CF0005D936D937C93139781E0DF01A15BBF4FB0
:105D00001D921D921D921C921397E15AFF4F91E034
:105D10009083DF91CF911F910F91FF90EF90DF90D3
:105D2000CF9008950F931F93CF93DF938C01D62FBD
:105D3000FC018589811109C0C80117DFC82FC8017E
:105D400004DFD11108C08C2F06C0C801FEDEC82FA9
:105D5000C8010BDFF6CFDF91CF911F910F9108950E
:105D6000CF93DF93EC01FC01E759FF4F81E0808383
:105D700039978081B297882341F080819181A281F7
:105D8000B3810196A11DB11D07C080819181A281BF
:105D9000B3810197A109B10980839183A283B38361
:105DA000FE01E459FF4F20813181DE01A659BF4F2A
:105DB000C9019595879520FD03C0ED91FC910DC01B
:105DC000FE01E80FF91F0190F081E02D2D913C912B
:105DD000E20FF31F0190F081E02D8C0F9D1F1995AC
:105DE0008F859889892B11F1FE01E059FF4F2081A1
:105DF0003181DE01A259BF4FC9019595879520FDDC
:105E000003C0ED91FC910DC0FE01E80FF91F019058
:105E1000F081E02D2D913C91E20FF31F0190F08174
:105E2000E02D8C0F9D1FDF91CF911994DF91CF91C1
:105E300008958F929F92AF92BF92CF92DF92EF928E
:105E4000FF920F931F93CF93DF93EC01FC01E15B73
:105E5000FF4F60817181828193810E94AC4C6B0104
:105E60007C0168A979A98AA99BA90E94AE4C9B01D3
:105E7000AC0160E074E284E799E40E949C4E4B011F
:105E80005C01FE01E55AFF4F60817181828193813F
:105E90000E94AC4C9B01AC01C501B4010E949C4E18
:105EA0004B015C018E010D5A1F4F20E030E040E0B5
:105EB0005FE30E940D4D9B01AC01C701B6010E943A
:105EC000384E0E94094FF801608371838283938367
:105ED000C95ADF4FA5019401C701B6010E94384E8F
:105EE0000E94094F688379838A839B83DF91CF91D6
:105EF0001F910F91FF90EF90DF90CF90BF90AF90E8
:105F00009F908F9008950F931F93CF93DF93FC0181
:105F1000E759FF4F20812223B9F07A970081118140
:105F200022813381389640815181628173810417C7
:105F300015072607370710F1EC01EEDDCE01DF91E2
:105F4000CF911F910F9175CFFC01E15AFF4F208136
:105F50002223A1F070970081118122813381349630
:105F60004081518162817381041715072607370725
:105F700028F0DF91CF911F910F91F2CEDF91CF9159
:105F80001F910F9108952F923F924F925F926F92BF
:105F90007F928F929F92AF92BF92CF92DF92EF92B9
:105FA000FF920F931F93CF93DF93CDB7DEB7629726
:105FB0000FB6F894DEBF0FBECDBF8C017C0126E486
:105FC000E20EF11CD7018C919801205A3F4FF80145
:105FD000EF59FF4F6F01A801425C5F4F4A011497D0
:105FE0001D01882341F0F80184A5D9018C9381E03B
:105FF000F60180832FC0DA014D915D916D917C9106
:10600000F10180819181A281B381BB24B3944817AF
:1060100059076A077B070CF0B12CF901B08277FFB2
:1060200007C070956095509541955F4F6F4F7F4FBA
:10603000B7FF07C0B095A095909581959F4FAF4F42
:10604000BF4F21E0481759076A077B070CF420E08F
:10605000D6012C93F40140815181628173814115F5
:1060600051056105710559F4F801848D958DA68D52
:10607000B78DE55AFF4F80839183A283B383F101EB
:1060800080819181A281B381F80142AC53AC64ACB0
:1060900075AC9801215A3F4F5901481659066A06B6
:1060A0007B0634F4481759076A077B077CF00AC05F
:1060B00084159505A605B7052CF484179507A60742
:1060C000B70724F0D7018C918823D9F0F50180819E
:1060D0008823B9F0D7018C91811105C0F701808127
:1060E00081110FC006C060E0C8011CDE8111F6CF2F
:1060F00017C0D6016C9181E06827C80113DE8823A0
:1061000079F0D5011C9260E0C8010CDE882309F407
:10611000C6C1F801FE961082118212821382BFC19D
:10612000D80194962D913D914D915C91979729833B
:106130003A834B835C8358962D913D914D915C91B0
:106140005B972D833E834F8358875C962D913D91BD
:106150004D915C915F9729873A874B875C87F10166
:1061600080819181A281B381F801FE96C080D180A7
:10617000E280F380F80142AD53AD64AD75ADED59E9
:10618000FF4F1082319610823801F5E66F0E711CB8
:10619000F301108298012A593F4FF901108232967B
:1061A00010824C015D01841A950AA60AB70AB7FE4F
:1061B00008C0B094A09490948094811C911CA11C60
:1061C000B11C481759076A077B072CF4C41AD50A73
:1061D000E60AF70A04C0C81AD90AEA0AFB0AD50176
:1061E000C401B595A795979587958D879E87AF87AD
:1061F000B88BD801A859BF4F1D01F7FC05C08C14FE
:106200009D04AE04BF044CF4F80100A0F1A1E02D00
:10621000FA8BE98B81E0D9011BC02D853E854F8526
:1062200058892C153D054E055F0508F454C0898139
:106230009A81AB81BC818C159D05AE05BF0564F4C8
:106240002D813E812F5F3F4F3A8B298B81E0D30117
:106250008C93F10180839EC0C701B6010E94AE4CB1
:106260002B013C0169817A818B819C810E94AE4C1B
:106270009B01AC01C301B2010E949C4E2B013C0169
:106280006D817E818F81988529853A854B855C85D6
:10629000621B730B840B950B0E94AE4C9B01AC01EF
:1062A000C301B2010E940D4D2B013C0169857A8525
:1062B0008B859C850E94AE4C9B01AC01C301B20151
:1062C0000E94384E0E94044F7A8B698B81E0F8015E
:1062D000ED59FF4F5CC0D501C40129813A814B8142
:1062E0005C81821B930BA40BB50BC816D906EA067A
:1062F000FB065CF42D813E812E5F3F4F3A8B298B4C
:1063000081E0F801EB59FF4F42C0C501B4016C199F
:106310007D098E099F090E94AE4C2B013C016981C9
:106320007A818B819C810E94AE4C9B01AC01C301A0
:10633000B2010E949C4E2B013C016D817E818F81B8
:10634000988529853A854B855C85621B730B840B88
:10635000950B0E94AE4C9B01AC01C301B2010E949F
:106360000D4D2B013C0169857A858B859C850E94AA
:10637000AE4C9B01AC01C301B2010E94384E0E9499
:10638000044F7A8B698B81E0F801EC59FF4F8083D1
:10639000D1018C93F80184818823B1F00E94742983
:1063A000D80112964D905C901397052C000C66084E
:1063B0007708DC01CB0184199509A609B709893E44
:1063C0009340A105B10568F4F801E55AFF4F29890A
:1063D0003A89C901A0E0B0E080839183A283B383AE
:1063E00092CE0E947429D80113967C936E931297D3
:1063F00084E294E00E94053B86E196E00E94053B22
:1064000060E070E0CB010E94513B8CE196E00E947D
:10641000053BC701B6010E94513B82E296E00E9413
:10642000053BC501B4010E94513B88E296E00E9401
:10643000053B4AE06D857E858F8598890E94063BE5
:106440008FE296E00E94053B69817A818B819C8175
:106450000E94513B85E396E00E94053B69857A8561
:106460008B859C850E94513B8BE396E00E94053B07
:106470006D817E818F8198850E94513B81E496E0F9
:106480000E94053B8EE496E00E94053B89899A892B
:106490000E94783B8CE993E00E94053B95CF629681
:1064A0000FB6F894DEBF0FBECDBFDF91CF911F9125
:1064B0000F91FF90EF90DF90CF90BF90AF909F90A3
:1064C0008F907F906F905F904F903F902F900895A6
:1064D0000F931F93FC01EA5BFF4F2081211110C035
:1064E0003897008111812281338134964081518116
:1064F00062817381041715072607370744F404C027
:10650000FC0124A5222319F01F910F9156CB1F9156
:106510000F913BCBFC0113821282148216821582EA
:1065200010861782128611861486138616861586A3
:10653000108A1786128A118A148A138ADC01A15ADA
:10654000BF4F1C9212AE13AE14AE15AE91971D92B2
:106550001D921D921C92139714961D921D921D92CE
:106560001C92139714961C925A961C9211961C9288
:1065700012961C9211961C9211961C9211961C92C6
:1065800011961C9211961C9211961C9211968DE1F7
:106590009DE211969C938E93129611961C921E92D8
:1065A000129689E19DE211969C938E931296119614
:1065B0001C921E92129685E19DE211969C938E93F9
:1065C000129611961C921E92129681E19DE28D9375
:1065D0009C93E858FF4F11821082089508956E34FD
:1065E00071050CF050C06B3471050CF08FC06C322B
:1065F000710554F5693271050CF088C06831710578
:1066000094F46F3071050CF081C06630710544F46C
:10661000623071050CF07AC0672B09F075C076C046
:106620006B5071096EC0623271053CF46F317105B7
:106630000CF06CC06951710964C064527109623018
:10664000710508F061C062C06A3371057CF467337C
:1066500071050CF05BC06D3271050CF455C06033F0
:1066600071050CF453C0635371094BC06434710558
:106670003CF4613471050CF049C06D53710941C09F
:10668000675471093EC066387105F4F463387105CA
:10669000ECF56237710564F46F367105BCF565364B
:1066A000710594F1683671058CF16956710929C03C
:1066B0006C37710534F46937710544F56357710916
:1066C00020C06D5771091DC0603D71057CF46D3CA3
:1066D0007105E4F46439710534F461397105B4F479
:1066E0006D5871090EC0695C71090BC06A3D710576
:1066F00034F4673D710554F4635D710902C06D5D4A
:1067000071096330710510F080E0089581E008950B
:106710000C9496470C9496470C9496470C94964785
:106720000C9496470C9496470C9496470C94964775
:106730000C9496470C9496470C9496478F929F9290
:10674000AF92BF92CF92DF92EF92FF920F931F937F
:106750000E94DD1660E070E046D2892BD1F40E94E1
:10676000DD161F921F9221E02F931F921F92812C02
:10677000912CA12CB12CC12CD12C76019701860132
:10678000B701A6010E941A0B0F900F900F900F9067
:106790000F9080E090E01F910F91FF90EF90DF90BD
:1067A000CF90BF90AF909F908F9008958F929F92BF
:1067B000AF92BF92CF92DF92EF92FF920F931F930F
:1067C0000E94DD1661E070E00ED2892BD1F40E94A8
:1067D000DD161F9221E02F931F921F921F92812C92
:1067E000912CA12CB12CC12CD12C760197018601C2
:1067F000B701A6010E941A0B0F900F900F900F90F7
:106800000F9080E090E01F910F91FF90EF90DF904C
:10681000CF90BF90AF909F908F900895EF92FF928E
:106820000F931F93CF93DF9300D01F92CDB7DEB7A6
:10683000FB0122A133A144A155A1068D178D298307
:106840003A834B835C830E941A097C01FC0182819C
:10685000938129813A814B815C818F30F7E29F07D8
:106860002CF40196F7019383828303C0F70113820E
:106870001282B801C70129833A834B835C83AFDE60
:1068800029813A814B815C818823A1F0F801EE0FC8
:10689000FF1FEE0FFF1FEA5AF84F20833183428318
:1068A0005383B801C7010E948808B801C7010E943C
:1068B000D70803C085ED94E0A8D6D2D80E94171B54
:1068C00080E090E00F900F900F900F90DF91CF91AC
:1068D0001F910F91FF90EF9008950F931F93CF9307
:1068E000DF930E941A098C01C0E0D0E0BE01C8010C
:1068F00076DE882321F0BE01C8010E94D7082196C8
:10690000C13ED10599F787E496E07FD60E948918A9
:106910000E94931780E090E0DF91CF911F910F913B
:1069200008958BE496E071D685E593E06ED60E94DB
:1069300089180E94931780E090E008950E948918BA
:10694000FC01148680E090E008958091A60B909160
:10695000A70B892BA1F480E790E00E940147FC017E
:10696000F9969C0123593F4FDF01D8971C92119251
:10697000E217F307C9F79093A70B8093A60B8091BA
:10698000A60B9091A70B08956F927F928F929F9282
:10699000AF92BF92CF92DF92EF92FF920F931F932D
:1069A000CF93DF93FB01E2A8F3A886A497A4A0A845
:1069B000B1A8C6A0D7A062A073A0068D178DC5DFB1
:1069C000EC019701A301B8010E94320AC501B4018C
:1069D0000E943C299701A601B801CE010E94320A0B
:1069E00080E090E0DF91CF911F910F91FF90EF90A9
:1069F000DF90CF90BF90AF909F908F907F906F90DF
:106A000008950F931F93CF93DF93FB0102A913A95E
:106A1000C68DD78D9ADFA801BE010E949B0980E038
:106A200090E0DF91CF911F910F9108951F93CF9325
:106A3000DF931F92CDB7DEB7FB0162A9168D698384
:106A400084DF6981812F0E94F52880E090E00F901B
:106A5000DF91CF911F910895EF92FF920F931F93B3
:106A6000CF93DF93FB01E2A8F3A802A113A1C68D87
:106A7000D78D6BDF9701A801BE010E94320A80E02A
:106A800090E0DF91CF911F910F91FF90EF900895CB
:106A900008950895089508950895CF93DF93EC0124
:106AA00088810E94D92721E0892B09F420E02C87D6
:106AB0008C810E94D92721E0892B09F420E02E87C0
:106AC0008E899F890197D1F48A810E94D92721E07C
:106AD000892B09F420E02D878E810E94D92721E09F
:106AE000892B09F420E02F879C858D85981749F024
:106AF0008E85821731F09A878B8703C08C858A87B1
:106B00002B87DF91CF9108950F93FC019285908799
:106B100083858187A689B789119721F4621721F0AF
:106B2000401711F06287438783858823D1F08285DF
:106B300091110AC08823A9F080899189A289B3891B
:106B40000197A109B10909C081110BC08089918900
:106B5000A289B3890196A11DB11D808B918BA28B57
:106B6000B38B0F910895CF93DF93FC01A489B5896E
:106B7000C08DD18D2089318942895389A03187E226
:106B8000B80759F01A161B0644F40E94004E20E183
:106B900037E240E050E00E94DA4DDE010E94004EF4
:106BA000DF91CF910895FC0181E090E0938F828F77
:106BB0001182108215821482108A118A128A138A15
:106BC000178A168A80E197E2958B848B128610864D
:106BD00014861586168617860895089508950895D3
:106BE0000895089508952F923F924F925F926F9269
:106BF0007F928F929F92AF92BF92CF92DF92EF924D
:106C0000FF920F931F93CF93DF93CDB7DEB7A39778
:106C10000FB6F894DEBF0FBECDBF9BA38AA31B01A6
:106C20000E94271D8AA19BA10E944C1B8AA19BA1A7
:106C30000E94562C8AA19BA10E945A2C21E0221668
:106C40003104C9F132E02316310409F466C021147D
:106C5000310409F095C0AAA0BBA040E1A40EB11C6C
:106C60008AA19BA182589E4F9E838D83EAA1FBA19E
:106C7000EA5BFD4F90819D87AAA1BBA1A959BD4F99
:106C8000B887AF83EAA1FBA1EF56FD4FF98BE88BE4
:106C90002AA13BA12D553D4F3D8B2C8B4AA15BA1D9
:106CA0004D515E4F5C874B878DE890E09B8B8A8BC4
:106CB000A5E1B0E062C0AAA0BBA0BAE8AB0EB11CCF
:106CC000EAA1FBA1E656FE4FFE83ED83EAA1FBA1FC
:106CD000E95BFD4F20812D874AA15BA145595D4F9E
:106CE00058874F838AA19BA18D569D4F998B888B86
:106CF000AAA1BBA1AC55BD4FBD8BAC8BEAA1FBA13A
:106D0000EB51FE4FFC87EB872EE830E03B8B2A8B64
:106D100046E150E05C834B8336C0AAA0BBA05CEF89
:106D2000A51A5EEFB50A8AA19BA18A549E4F9E8345
:106D30008D83EAA1FBA1E85BFD4F90819D87AAA10D
:106D4000BBA1A159BD4FB887AF83EAA1FBA1EB5608
:106D5000FD4FF98BE88B2AA13BA12B553D4F3D8B75
:106D60002C8B4AA15BA149515E4F5C874B878FE812
:106D700090E09B8B8A8BA7E1B0E0BC83AB8303C020
:106D800080E596E00CC0C5010E94B52D811105C0BB
:106D9000C5010E94A52D882369F081EE96E035D4C7
:106DA0000E94891881E090E0909345078093440702
:106DB00090E0C8C384E294E028D48FE796E025D41D
:106DC000D5018C9163D487E197E01FD48CE993E0DF
:106DD0001CD481E090E0EB85FC859183808341E0C9
:106DE00050E0B5018AA19BA10E94E118C5010E9453
:106DF000072ED5019C968C918501005A1F4F882340
:106E000039F0C5010E94DD2D81E0F801808305C0C5
:106E1000C5010E94C52DD8011C928D819E81A3DEE3
:106E2000F501FE966083718382839383EF81F885F9
:106E30001082118212821382EAA1FBA1E959FD4F4F
:106E40001082118212821382EAA1FBA1E559FD4F43
:106E50001082118212821382EAA1FBA1E159FD4F37
:106E6000108211821282138286E090E0AB85BC858D
:106E70008D939C9346E050E0B5018AA19BA10E94AE
:106E8000E11841E050E0B5018AA19BA10E94C6181B
:106E9000412C512C320143948AA19BA1820D931D58
:106EA000FC01ED55FD4FFF87EE874101880C991CD1
:106EB000880C991CC40189569D4F2AA13BA1280F1B
:106EC000391F3F8B2E8BC101875A9E4F880F991F08
:106ED0004AA15BA1480F591F5B8F4A8FC4018B5792
:106EE0009D4FAAA1BBA1A80FB91FBD8FAC8FF40104
:106EF000E758FD4FFF8FEE8F8AA19BA1880D991D4A
:106F00009C01205F3D4F3A872987AE85BF858C91D4
:106F10008823B1F0A40149595D4FEAA1FBA14E0FAE
:106F20005F1FCE88DF88EA8CFB8C0C8D1D8D2E8D2B
:106F30003F8D2E0F3F1F6D817E81C5010E949A2BD0
:106F400088EA9BE00E94E4241816190624F01A82AD
:106F5000198210E01DC088EA9BE00E94C2248F7D48
:106F600085349105A1F782E095E04FD30E948918FE
:106F700021E0DC011C962C9382E693E046D30E942C
:106F800089180E949317E1E0F0E0FA83E98311E0A9
:106F9000C5010E94B52D8111C4C2C5010E94A52D55
:106FA0008111BFC21111BDC2A889B9896D917C91AF
:106FB000072E000C880B990B0E94AE4C9B01AC0174
:106FC000EF81F88560817181828193810E94A84C54
:106FD00087FFA7C2C5010E94B02EE985FA852081EE
:106FE00031814281538160E573EC80E090E00E9442
:106FF000DA4DC9010E943129A985BA852D913D91AB
:107000004D915C91A3E0B0E00E94F64D9B01AC0174
:10701000C301B2010E94DA4D672B682B692B39F44A
:107020008EE593E0F2D20E9489180E949317C50161
:107030000E948C2DA985BA852D913D914D915C9131
:1070400060E573EC80E090E00E94DA4DC9010E9497
:107050003129BFEF4B1A5B0A6B0A7B0AE981FA817F
:10706000EF2B09F452CF21E030E03A83298342E04C
:1070700050E0B5018AA19BA10E94C61884E294E069
:10708000C4D28FE796E0C1D2D5018C91FFD286E8B9
:1070900096E0BBD28CE993E0B8D2E981FA81EF2B7C
:1070A000D1F489E996E0B1D28EE496E0AED281EDDA
:1070B00094E0ABD28B819C811BD38EE496E0A5D269
:1070C00083ED94E0A2D2FD858F2F90E011D30E9432
:1070D00089180E9493178AA19BA10E94562C8AA10D
:1070E0009BA10E945A2C84E294E08FD28FE796E015
:1070F0008CD2D5018C91CAD28DE996E086D28CE9EA
:1071000093E083D2EF81F88510821182128213827C
:10711000D5019C968C918501005A1F4F882331F030
:10712000C5010E94C52DF801108206C0C5010E944C
:10713000DD2D81E0D8018C938D819E8114DDF501D8
:10714000FE966083718382839383EAA1FBA1E95950
:10715000FD4F1082118212821382EAA1FBA1E55930
:10716000FD4F1082118212821382EAA1FBA1E15924
:10717000FD4F10821182128213828D819E81F3DC79
:107180006E8B7F8B888F998F412C512C32014394C9
:107190008AA19BA1820D931DFC01ED55FD4FFB8F34
:1071A000EA8F9101220F331F220F331F3C832B8361
:1071B000C90189569D4F4AA15BA1480F591F5D8F98
:1071C0004C8FC101875A9E4F880F991FAAA1BBA15E
:1071D000A80FB91FBF8FAE8FC9018B579D4FEAA172
:1071E000FBA1E80FF91FF9A3E8A3C9012AA13BA15C
:1071F000820F931FAC01405F5D4F5F874E87920106
:10720000215031093A872987490149815A81452B03
:1072100009F0C7C0AA8DBB8D8C918823C9F02B8142
:107220003C8127583D4FEAA1FBA12E0F3F1F4B8108
:107230005C8149595D4F4E0F5F1FCC8CDD8CEE8C0D
:10724000FF8C08A119A16D817E81C5010E949A2B36
:1072500088EA9BE00E94E4241816190614F010E056
:107260001DC088EA9BE00E94C2248F7D8534910571
:10727000B1F782E095E0C9D10E94891821E0DC01D4
:107280001C962C9382E693E0C0D10E9489180E943C
:107290009317E1E0F0E0FA83E98311E029853A856C
:1072A0002A30310538F4AF81B8851D921D921D92A8
:1072B0001C921397BD85C501B1113FC10E94A52D38
:1072C00081116BC0112319F089849A8466C0E88902
:1072D000F98960817181072E000C880B990B0E943F
:1072E000AE4C9B01AC01AF81B8856D917D918D91C4
:1072F0009C910E94A84C87FFE7CFC5010E94B02E49
:10730000EE85FF85208131814281538160E573ECF8
:1073100080E090E00E94DA4DC9010E943129AE85DB
:10732000BF852D913D914D915C91A3E0B0E00E940D
:10733000F64D9B01AC01C301B2010E94DA4D672BEF
:10734000682B692B91F48EE593E05FD10E94891838
:107350000E94931784E294E058D181EB96E055D1D6
:10736000C201C6D18CE993E050D1C5010E948C2D99
:10737000EE85FF85208131814281538160E573EC88
:1073800080E090E00E94DA4DC9010E943129FFEFB0
:107390004F1A5F0A6F0A7F0A32CF8FEB96E035D122
:1073A00004C081E090E09A83898384E294E02DD147
:1073B0008FE796E02AD1D5018C9168D183ED96E0D4
:1073C00024D18CE993E021D18D819E81CCDBEC89A5
:1073D000FD89EF2BA1F0DC01CB012E893F89488D7F
:1073E000598D821B930BA40BB50BB7FF07C0B0954B
:1073F000A095909581959F4FAF4FBF4F4C0149810C
:107400005A81452BF9F489E996E0FFD08EE496E0A5
:10741000FCD081ED94E0F9D08A899B8969D18EE412
:1074200096E0F3D083ED94E0F0D0B401092C000C89
:10743000880B990B0E94AE4C42E05FD10E948918E4
:107440000E94931785E090E0AB85BC858D939C935B
:1074500045E050E0B5018AA19BA10E94E118C50159
:107460000E94F52D8AA19BA10E94562C8AA19BA166
:107470000E945A2CB1E02B163104A9F0E2E02E163E
:10748000310401F1232861F50E948918C401990C87
:10749000AA0BBB0B80934A0790934B07A0934C0712
:1074A000B0934D071DC00E948918C401990CAA0B06
:1074B000BB0B80934E0790934F07A0935007B09358
:1074C00051070EC00E948918C401990CAA0BBB0B6E
:1074D0008093520790935307A0935407B093550796
:1074E0000E9489180E94E617AB85BC851D921C92EC
:1074F00040E050E0B5018AA19BA10E94E11840E064
:1075000050E0B5018AA19BA10E94C6180E9489186B
:10751000E981FA81F0934507E093440789819A81D4
:1075200011C08FEB96E071D0C5010E94A52D882374
:1075300009F49DCDB1E0BD879ACD0E94B52D811192
:10754000C3CEC0CEA3960FB6F894DEBF0FBECDBF9C
:10755000DF91CF911F910F91FF90EF90DF90CF902F
:10756000BF90AF909F908F907F906F905F904F9063
:107570003F902F900895CF93DF93FC01EA52FE4F86
:10758000408151814115510559F1EC01C652DE4F40
:10759000288139818E529E4F24173507C8F4FC018B
:1075A00080819181009761F0FC01E20FF31F8081DF
:1075B0008A3041F08D3029F48CE993E026D002C066
:1075C00080E064D08881998101969983888308C07E
:1075D00040E050E06EE973E00E943C271982188277
:1075E000DF91CF910895009769F0FC010190002090
:1075F000E9F73197AF01481B590BBC0188EA9BE0C2
:107600000C94842480E090E00895EDCF8F929F92B7
:10761000AF92BF920F931F93CF93DF93CDB7DEB797
:10762000A1970FB6F894DEBF0FBECDBF19A24230AE
:1076300008F44AE08E010F5D1F4F842E912CA12C7F
:10764000B12CA50194010E94064EE62FB901CA0192
:1076500001501109EA3014F4E05D01C0E95CD80181
:10766000EC93232B242B252B61F7C801BCDFA196BB
:107670000FB6F894DEBF0FBECDBFDF91CF911F9143
:107680000F91BF90AF909F908F900895E091A80BBD
:10769000F091A90B0190F081E02D682F88EA9BE022
:1076A0001994CF92DF92EF92FF92CF93DF9397FFDF
:1076B00017C06B017C018DE2E9DFEC0166277727BB
:1076C000CB016C197D098E099F094AE09FDF8C0F61
:1076D0009D1FDF91CF91FF90EF90DF90CF900895A5
:1076E0004AE0DF91CF91FF90EF90DF90CF908ECF67
:1076F000BC01990F880B990BD4CF4F925F926F9278
:107700007F928F929F92AF92BF92CF92DF92EF9231
:10771000FF926B017C01B42E9B01AC010E94394F9A
:10772000882319F086E397E027C026013701E89403
:1077300077F82FEF3FEF4FE75FE7C301B2010E94F9
:10774000394F81110DC02FEF3FEF4FE75FE7C301C6
:10775000B2010E94A84C18161CF48AE397E00CC0F2
:107760002FEF3FEF4FE75FE4C701B6010E94354FAF
:1077700018167CF48EE397E0FF90EF90DF90CF90A7
:10778000BF90AF909F908F907F906F905F904F9041
:107790002ACF2FEF3FEF4FE75FECC701B6010E9402
:1077A000A84C87FDE7CF20E030E0A901C701B60172
:1077B0000E94A84C87FF08C08DE268DF4C01F7FAF1
:1077C000F094F7F8F09402C0812C912CA12C60E089
:1077D00070E080E09FE3AB1441F020E030E040E255
:1077E00051E40E949C4EA394F6CF9B01AC01C701CB
:1077F000B6010E94384E2B013C010E94094F6B01DB
:107800007C010E94AC4C9B01AC01C301B2010E94FF
:10781000374E2B013C014AE0C701B601F7DE7C017F
:10782000E80CF91CBB2021F08EE230DFE80EF91ED7
:10783000DB2CDD2019F120E030E040E251E4C3010F
:10784000B2010E940D4D2B013C010E94094F4B01DA
:10785000A12CB12C4AE0C501B401D8DEE80EF91E16
:10786000C501B4010E94AC4C9B01AC01C301B20143
:107870000E94374E2B013C01DA94DBCFC701FF9009
:10788000EF90DF90CF90BF90AF909F908F907F90C0
:107890006F905F904F900895789484B5826084BD16
:1078A00084B5816084BD85B5826085BD85B5816004
:1078B00085BD80916E00816080936E001092810082
:1078C000809181008260809381008091810081603D
:1078D00080938100809180008160809380008091FE
:1078E000B10084608093B1008091B000816080938A
:1078F000B00080919100826080939100809191000E
:1079000081608093910080919000816080939000CD
:107910008091A10082608093A1008091A10081608C
:107920008093A1008091A00081608093A00080914D
:1079300021018260809321018091210181608093E7
:1079400021018091200181608093200180917A0043
:10795000846080937A0080917A00826080937A00BC
:1079600080917A00816080937A0080917A008068AB
:1079700080937A001092C10061E08AE10E94F528AC
:1079800061E08BE10E94F52861E089E10E94F52821
:1079900061E08FE00E94F52861E08EE10E94F52809
:1079A00061E08EE00E94F52862E085E40E94F528FF
:1079B00062E084E40E94F52862E080E10E94F528FC
:1079C00062E081E10E94F52861E080E20E94F528F2
:1079D00061E081E20E94F52861E08FE10E94F528D4
:1079E00062E083E40E94F52862E082E40E94F528C8
:1079F00062E087E10E94F52862E088E10E94F528B4
:107A000061E083E20E94F52861E084E20E94F528AB
:107A100061E082E20E94F52862E081E40E94F5289C
:107A200062E080E40E94F52862E08DE10E94F52882
:107A300062E08CE10E94F52861E088E20E94F5286E
:107A400061E089E20E94F52861E085E20E94F52864
:107A500061E085E20E94012861E08DE00E94F52846
:107A600061E089E00E94F52861E088E00E94F52845
:107A700061E087E00E94F52861E08AE00E94F52835
:107A800061E08CE00E94F52862E08FE30E94F52817
:107A900062E08BE30E94F52861E084E00E94F52813
:107AA00061E085E00E94F52861E086E00E94F5280B
:107AB00061E087E00E94F52861E089E10E940128E9
:107AC00061E08EE00E94012861E08FE10E940128C0
:107AD00061E082E20E940128E091B80BF091B90BBD
:107AE00082E08083E091B40BF091B50B1082E091BD
:107AF000B60BF091B70BD0E1D0831092C00BE091A0
:107B0000BC0BF091BD0B86E08083E091BA0BF09145
:107B1000BB0B808180618083E091BA0BF091BB0B3D
:107B2000808188608083E091BA0BF091BB0B8081EB
:107B300080688083E091BA0BF091BB0B80818F7DD0
:107B4000808364E670E080E090E00E943C290E941F
:107B5000DD160E948C130E94302D0E94171B0E947C
:107B6000742960937E0B70937F0B8093800B9093AE
:107B7000810B82ED97E09093430780934207C1E029
:107B8000C0936F00D093810010928000C093DC0AF4
:107B900080E092E09093DB0A8093DA0A909387006A
:107BA0008093860081E18093810010928100109281
:107BB0008500109284008091DC0A806180938100AE
:107BC0000E94742960937A0B70937B0B80937C0BDB
:107BD00090937D0B0E9474296093820B7093830BAA
:107BE0008093840B9093850B0E94742960937E0B85
:107BF00070937F0B8093800B9093810B0E941A09E6
:107C000080915E0790915F07A0916007B091610736
:107C10000197A105B10579F40E941A098091A60780
:107C20009091A707A091A807B091A9070197A10576
:107C3000B10509F4C9C70E941A0980915E079091A5
:107C40005F07A0916007B09161070197A105B10599
:107C500079F40E941A098091A2079091A307A0913C
:107C6000A407B091A5070197A105B10509F4CAC7FA
:107C70000E941A0980915E0790915F07A0916007AA
:107C8000B09161070197A105B10579F40E941A0925
:107C900080919E0790919F07A091A007B091A107A6
:107CA0000197A105B10509F4CCC780E893E0ADDCEC
:107CB0008FE7282E82E0382E95E7A92E92E0B92E84
:107CC0000E9474296093820B7093830B8093840BC2
:107CD0009093850B00917E0B10917F0B2091800B70
:107CE0003091810B601771078207930748F4609306
:107CF0007E0B70937F0B8093800B9093810B2CC035
:107D0000DC01CB01801B910BA20BB30B883E93408F
:107D1000A105B10508F108511C4F2F4F3F4F0093AB
:107D20007E0B10937F0B2093800B3093810B0E946E
:107D3000302DEC010E94022BCE010C960E94022BEA
:107D4000CE0148960E94022BCE0184960E94022BFF
:107D5000CE01C0960E94022B88EA9BE00E94E42498
:107D6000892B09F4BCC50E94742960937A0B709327
:107D70007B0B80937C0B90937D0B88EA9BE00E94A9
:107D8000C2248093790B982F9F7D953479F02091B0
:107D9000770B3091780BF901EB5BF44F80832F5F09
:107DA0003F4F3093780B2093770B06C00E948918C1
:107DB00021E0DC011C962C938091770B9091780B3D
:107DC0008133910564F02AE02093790BFC01EB5B91
:107DD000F44F208301969093780B8093770B8091DA
:107DE000790B2091770B3091780B8A3039F4C901E7
:107DF0000197A2E1BBE0E5E4FBE004C022333105DA
:107E0000B4F76DC5AF0145545B40481759071CF4E2
:107E100041914D93F7CFFC01EE5EF44F108222307A
:107E200031050CF458C581E193E0EFDB8EE496E078
:107E3000ECDB8FE993E0E9DB82E19BE0E6DB8FE9B5
:107E400093E0E3DB8CE993E0E0DB8AE390E0D9D7D1
:107E5000EC011A821B821C821D821E821F821886E0
:107E600019861A861B861C861D861E861F86188A02
:107E7000198A1A8A1B8A1C8A1D8A1E8A1F8A188ED2
:107E8000198E1A8E1B8E1C8E1D8E1E8E1F8E18A292
:107E900019A21AA21BA21CA21DA21EA21FA218A6F2
:107EA00019A61AA61BA61CA61DA61EA61FA618AAC2
:107EB00019AA1AAA1BAA1CAA1DAA1EAA1FAA18AE92
:107EC00019AE68E072E082E19BE00E9431488C01CB
:107ED000FC0180818654823008F027C161EA73E09A
:107EE000C8010E943950892B09F4D3C064EA73E0B9
:107EF000C8010E943950892B09F4CBC068EA73E0AD
:107F0000C8010E943950892B09F4C6C06BEA73E09E
:107F1000C8010E943950892B09F4BEC06FEA73E092
:107F2000C8010E943950892B09F4B9C063EB73E092
:107F3000C8010E943950892B09F4B4C067EB73E083
:107F4000C8010E943950892B09F4ACC06AEB73E078
:107F5000C8010E943950892B09F4A7C06EEB73E069
:107F6000C8010E943950892B09F4A2C062EC73E069
:107F7000C8010E943950892B09F49DC066EC73E05A
:107F8000C8010E943950892B09F498C06AEC73E04B
:107F9000C8010E943950892B09F493C06EEC73E03C
:107FA000C8010E943950892B09F48EC062ED73E03C
:107FB000C8010E943950892B09F489C066ED73E02D
:107FC000C8010E943950892B09F484C06AED73E01E
:107FD000C8010E943950892B09F47FC06EED73E00F
:107FE000C8010E943950892B09F47AC062EE73E00F
:107FF000C8010E943950892B09F475C066EE73E000
:10800000C8010E943950892B09F470C06AEE73E0F0
:10801000C8010E943950892B09F46BC06EEE73E0E1
:10802000C8010E943950892B09F466C062EF73E0E1
:10803000C8010E943950892B09F461C066EF73E0D2
:10804000C8010E943950892B09F45CC06AEF73E0C3
:10805000C8010E943950892B09F457C06EEF73E0B4
:10806000C8010E943950892B09F452C062E074E0C3
:10807000C8010E943950892B09F44DC066E074E0B4
:10808000C8010E943950892B09F448C08FEF9FEF37
:1080900047C080E090E044C081E090E041C08CE1C6
:1080A00090E03EC08DE690E03BC08FE690E038C0A7
:1080B00080E790E035C081E790E032C082E790E051
:1080C0002FC083E790E02CC084E790E029C088E7C8
:1080D00090E026C089E790E023C08AE790E020C0C6
:1080E00083E890E01DC084E890E01AC08DE890E03D
:1080F00017C08EE890E014C08FE890E011C080E9CE
:1081000090E00EC081EA90E00BC085EB90E008C0E3
:1081100086EB90E005C087EB90E002C088EB90E032
:108120009093010280930002BBC08FEF9FEF90936A
:10813000010280930002B8C0D8018C91883539F4CF
:10814000C80101968BD76A837B838C839D83F8015A
:108150008081893539F4C801019680D76E837F8389
:1081600088879987D8018C918A3539F4C80101969E
:1081700075D76A877B878C879D87F80180818134DA
:1081800049F4C80101966AD70E94044F6E877F8721
:10819000888B998BD8018C91823449F4C80101965F
:1081A0005DD70E94044F6A8B7B8B8C8B9D8BF80173
:1081B0008081833449F4C801019650D70E94044F4E
:1081C0006E8B7F8B888F998FD8018C91833539F492
:1081D000C801019643D76A8F7B8F8C8F9D8FF801E2
:1081E0008081803549F4C801019638D70E94044F38
:1081F0006E8F7F8F88A399A3D8018C91863549F41F
:10820000C80101962BD70E94044F6AA37BA38CA3BD
:108210009DA3F8018081873549F4C80101961ED7D6
:108220000E94044F6EA37FA388A799A7D8018C91C1
:10823000853449F4C801019611D70E94044F6AA7FA
:108240007BA78CA79DA7F8018081843549F4C801DC
:10825000019604D70E94044F6EA77FA788AB99AB05
:10826000D8018C918D3449F4C8010196F7D60E944B
:10827000044F6AAB7BAB8CAB9DABF8018081813541
:1082800049F4C8010196EAD60E94044F6EAB7FAB59
:1082900088AF99AF6AE074E080E090E0E2D68C01AC
:1082A0000115110509F048CF0E948918DC011C96C0
:1082B0001C910E941A0940906A0750906B076090C9
:1082C0006C0770906D07CEA8DFA8E8ACF9AC0E94EF
:1082D0008918C0924607D0924707E0924807F0926B
:1082E0004907809100029091010299249394823071
:1082F000910538F09C012F5631092630310508F0E0
:10830000912C112371F08D36910559F09C0128575D
:1083100031092330310528F0855B9109039708F076
:10832000D0C20E941A0980915E0790915F07A091C8
:108330006007B09161070197A105B10529F0992067
:1083400019F08DEF92E0BFC2209719F489EF92E007
:10835000BAC2E0900002F0900102BFEFEB16FB06FC
:10836000A9F3E114F104B9F48091DD0A9091DE0AD9
:10837000892B61F482E090E044D521E132E0FC01F8
:10838000318320839093DE0A8093DD0A0091DD0A19
:108390001091DE0A6EC0FCE1EF16F104B9F4809191
:1083A000DF0A9091E00A892B61F482E090E029D500
:1083B0002BE132E0DC012D933C939093E00A809313
:1083C000DF0A0091DF0A1091E00A53C0BDE6EB1608
:1083D000F104B9F48091E10A9091E20A892B61F4E9
:1083E00082E090E00ED525E232E0FC01318320836B
:1083F0009093E20A8093E10A0091E10A1091E20A67
:1084000053C0FFE6EF16F104B9F48091E30A9091AE
:10841000E40A892B61F482E090E0F3D42FE232E0A9
:10842000DC012D933C939093E40A8093E30A00913E
:10843000E30A1091E40A53C000E010E0B0E7EB1645
:10844000F104B9F48091E50A9091E60A892B61F470
:1084500082E090E0D6D429E332E0FC01318320832E
:108460009093E60A8093E50A0091E50A1091E60AE6
:108470006CC0F1E7EF16F104B9F48091E70A90912E
:10848000E80A892B61F482E090E0BBD423E432E077
:10849000DC012D933C939093E80A8093E70A0091C6
:1084A000E70A1091E80A6CC0B2E7EB16F104B9F4E0
:1084B0008091E90A9091EA0A892B61F482E090E0C8
:1084C000A0D42DE432E0FC01318320839093EA0AAA
:1084D0008093E90A0091E90A1091EA0A6AC0F3E779
:1084E000EF16F104B9F48091EB0A9091EC0A892B14
:1084F00061F482E090E085D427E532E0DC012D9341
:108500003C939093EC0A8093EB0A0091EB0A109154
:10851000EC0A68C0B4E7EB16F104B9F48091ED0AF7
:108520009091EE0A892B61F482E090E06AD421E612
:1085300032E0FC01318320839093EE0A8093ED0AB0
:108540000091ED0A1091EE0A68C0F8E7EF16F10409
:10855000B9F48091EF0A9091F00A892B61F482E0DE
:1085600090E04FD42BE632E0DC012D933C939093C6
:10857000F00A8093EF0A0091EF0A1091F00A68C0A8
:10858000B9E7EB16F104A9F48091F10A9091F20A8F
:10859000892B51F482E090E034D4FC01B182A082B6
:1085A0009093F20A8093F10A0091F10A1091F20A75
:1085B0006AC0FAE7EF16F104A9F48091F30A9091EA
:1085C000F40A892B51F482E090E01BD4DC012D9257
:1085D0003C929093F40A8093F30A0091F30A10916D
:1085E000F40A6CC0BDE8EB16F104B9F48091F50A09
:1085F0009091F60A892B61F482E090E002D429E898
:1086000032E0FC01318320839093F60A8093F50ACF
:108610000091F50A1091F60A6CC03EE8E316F104E9
:10862000B9F48091F70A9091F80A892B61F482E0FD
:1086300090E0E7D3E3E9F2E0DC01ED93FC93909363
:10864000F80A8093F70A0091F70A1091F80A6CC0B3
:10865000FFE8EF16F104B9F48091F90A9091FA0A53
:10866000892B61F482E090E0CCD3EDE9F2E0DC010B
:10867000ED93FC939093FA0A8093F90A0091F90A1A
:108680001091FA0A6CC0F0E9EF16F104B9F4809188
:10869000FB0A9091FC0A892B61F482E090E0B1D34F
:1086A000E7EAF2E0DC01ED93FC939093FC0A8093FF
:1086B000FB0A0091FB0A1091FC0A6CC0F1EAEF166C
:1086C000F104B9F48091FD0A9091FE0A892B61F4BE
:1086D00082E090E096D3E1EBF2E0DC01ED93FC93D5
:1086E0009093FE0A8093FD0A0091FD0A1091FE0A04
:1086F0006BC0F5EBEF16F104B9F48091FF0A90918D
:10870000000B892B61F482E090E07BD3EBEBF2E08D
:10871000DC01ED93FC939093000B8093FF0A009192
:10872000FF0A1091000B50C0F6EBEF16F104B9F4FC
:108730008091010B9091020B892B61F482E090E013
:1087400060D3E5ECF2E0DC01ED93FC939093020B37
:108750008093010B0091010B1091020B35C0F7EBD8
:10876000EF16F104B9F48091030B9091040B892B5F
:1087700061F482E090E045D3EFECF2E0DC01ED93B0
:10878000FC939093040B8093030B0091030B1091C7
:10879000040B1AC0F8EBEF16F104B1F48091050B4D
:1087A0009091060B892B61F482E090E02AD3E3EEEE
:1087B000F2E0DC01ED93FC939093060B8093050BA4
:1087C0000091050B1091060B0115110589F489EF35
:1087D00092E00E94053B0E9489180E9493178EE048
:1087E00094E00E94F33A8CE993E00E94F33A71C05E
:1087F00085EF92E00E94053B0E9489180E94931722
:108800000E9489181092450710924407E12CF12C20
:10881000FFEFEF1AFF0A21E0E216F10441F081EFC9
:1088200092E00E94053B0E9489180E949317D8018C
:10883000ED91FC910480F581E02DBE01C8011995F0
:108840000E948918C0904407D09045070E9489185B
:10885000FC018485E114F104D9F281110AC0E41409
:10886000F5043CF4C114D10421F0F2E0CF16D10498
:1088700079F688EA9BE00E94E424181619062CF485
:1088800088EA9BE00E94C224F4CFCD2809F4FBC102
:10889000992009F4F5C10E941A0980916607909108
:1088A0006707A0916807B09169070197A105B10515
:1088B00009F0E6C10E94891821E0DC011C962C9386
:1088C000DFC181E093E00E94053B0E9489180E946D
:1088D0009317CE012BD31092780B1092770B8091C7
:1088E000110B811170C00E948918FC0184858823B6
:1088F00009F469C00E94DD16EC01FC01EE53FD4F46
:10890000108240960E94F52DCE0186579F4F0E94FF
:10891000F52DCE018C5F9E4F0E94F52D0E94A5344F
:108920007C018C01075C1F4FC1E0D0E06801F8E3D7
:10893000CF1AD108D6018C918823D9F084E294E033
:108940000E94053B88E294E00E94053BCE010E9414
:10895000783B8CE993E00E94053B60E08C2F0E94FD
:10896000012840E050E0BE01C7010E949B09F601CA
:108970001082D8018C918823F9F084E294E00E945F
:10898000053B8FE394E00E94053BCE010E94783BBB
:108990008CE993E00E94053B61E08C2F0E94F52852
:1089A00060E08C2F0E94012841E050E0BE01C70129
:1089B0000E949B09F801108221960F5F1F4FC5335B
:1089C000D10509F0B3CF0E948918DC011C968C9167
:1089D0008093110BC0910F0BD091100B0E941A09BC
:1089E000FC0182819381C817D90799F00E941A0966
:1089F000DC0112968D919C9113979093100B8093AC
:108A00000F0B0E94DD160E948C130E94302D0E94D5
:108A1000171B0E94742960930B0B70930C0B8093AF
:108A20000D0B90930E0B00917A0B10917B0B209104
:108A30007C0B30917D0B601771078207930708F458
:108A4000B6C0DC01CB01801B910BA20BB30B8938A4
:108A50009341A105B10508F4B4C00E948918DC0156
:108A60001C968C91882319F08DE093E002C089E078
:108A700093E00E94053B0E9489180E9493170E9470
:108A8000DD16EC01FC01ED55FD4F8081882341F09E
:108A9000CE0182589E4F0E94B3356B017C0107C006
:108AA000FE01E25BFF4FC080D180E280F3800E9434
:108AB0008918C0924A07D0924B07E0924C07F09277
:108AC0004D07FE01EC55FD4F8081882341F0CE011A
:108AD00086569E4F0E94B3356B017C0107C0FE0194
:108AE000E853FF4FC080D180E280F3800E94891854
:108AF000C0924E07D0924F07E0925007F092510774
:108B0000FE01EB55FD4F8081882341F0CE018A5450
:108B10009E4F0E94B3356B017C0106C0CE5BDE4FD9
:108B2000C880D980EA80FB800E948918C0925207D1
:108B3000D0925307E0925407F09255070E9489188B
:108B40000E94E6170E94DD160E9470190E94891883
:108B50000E94D01A0E9489180E94A5170E941A0923
:108B600080915E0790915F07A0916007B0916107C7
:108B70000197A105B10541F085E093E00E94053B16
:108B80000E9489180E9493178091070B9091080BFF
:108B9000A091090BB0910A0B0196A11DB11D809304
:108BA000070B9093080BA093090BB0930A0B0E943C
:108BB000742960937A0B70937B0B80937C0B90935A
:108BC0007D0B0E9481257CC885E594E00E94053BD1
:108BD0000E94DD16CF931F921F921F921F92812C2D
:108BE000912CA12CB12CC12CD12C7601970186019E
:108BF000B701A6010E941A0B0F900F900F900F90D3
:108C00000F9019C88DE694E00E94053B0E94DD1686
:108C10001F9221E02F931F921F921F92812C912C63
:108C2000A12CB12CC12CD12C760197018601B70162
:108C3000A6010E941A0B0F900F900F900F900F90AB
:108C400017C885E894E00E94053B0E94DD161F923C
:108C50001F9221E02F931F921F92812C912CA12C07
:108C6000B12CC12CD12C760197018601B701A60148
:108C70000E941A0B0F900F900F900F900F9015C835
:108C800089EE92E002C08DEE92E00E94053B0E94C8
:108C900089180E9493170E94891810924607109213
:108CA0004707109248071092490713CE8091450C50
:108CB0009091460C3BC11092AB0B1092AA0B88EE20
:108CC00093E0A0E0B0E08093AC0B9093AD0BA09349
:108CD000AE0BB093AF0B8AE693E09093A90B809311
:108CE000A80B85EC90E09093B50B8093B40B84ECCB
:108CF00090E09093B70B8093B60B80EC90E090934C
:108D0000B90B8093B80B81EC90E09093BB0B8093F0
:108D1000BA0B82EC90E09093BD0B8093BC0B86EC79
:108D200090E09093BF0B8093BE0B1092C10B1092FA
:108D3000C20B1092C30B1092C40B82E090E061D082
:108D40002CE733E0FC013183208390934C0C80931B
:108D50004B0C6EE973E085E49CE00E9466278091ED
:108D6000DD0C803320F09FEF9093DE0C11C08093D8
:108D7000DE0C282F30E0F901EE0FFF1F2E0F3F1FF2
:108D8000F901E35BF34F28EB3BE0328321838F5FF4
:108D9000803390F48093E10C282F30E0F901EE0F3E
:108DA000FF1F2E0F3F1FF901E35BF34F28EB3BE062
:108DB000328321838F5F03C09FEF9093E10C8093F8
:108DC000DD0C0895EF920F931F93CF93DF93E8018B
:108DD00047FD02C034E001C034E1E42F440FFF0B33
:108DE000F7FF03C0F195E195F109E32E022F2E2F35
:108DF000AE01B3D1CE01DF91CF911F910F91EF90D2
:108E00000895CF93DF938230910510F482E090E0D3
:108E1000E091E80CF091E90C20E030E0C0E0D0E017
:108E2000309711F14081518148175907C0F0481718
:108E3000590761F482819381209719F09B838A837B
:108E40002BC09093E90C8093E80C26C021153105C6
:108E500019F04217530718F49A01BE01DF01EF0120
:108E60000280F381E02DDCCF2115310509F1281BAB
:108E7000390B2430310590F412968D919C91139703
:108E80006115710521F0FB019383828304C09093E7
:108E9000E90C8093E80CFD01329644C0FD01E20F1D
:108EA000F31F81939193225031092D933C933AC043
:108EB0002091E60C3091E70C232B41F42091040221
:108EC000309105023093E70C2093E60C20910202CA
:108ED000309103022115310541F42DB73EB7409181
:108EE000060250910702241B350BE091E60CF0912D
:108EF000E70CE217F307A0F42E1B3F0B28173907E6
:108F000078F0AC014E5F5F4F2417350748F04E0FE5
:108F10005F1F5093E70C4093E60C8193919302C03E
:108F2000E0E0F0E0CF01DF91CF9108950F931F9320
:108F3000CF93DF93009709F48CC0FC013297138222
:108F400012820091E80C1091E90C0115110581F4D1
:108F500020813181820F931F2091E60C3091E70C24
:108F60002817390779F5F093E70CE093E60C71C008
:108F7000D80140E050E0AE17BF0750F412962D9193
:108F80003C911397AD012115310509F1D901F3CFBA
:108F90009D01DA013383228360817181860F971FDF
:108FA0008217930769F4EC0128813981260F371F56
:108FB0002E5F3F4F318320838A819B8193838283FD
:108FC000452B29F4F093E90CE093E80C42C013968A
:108FD000FC93EE931297ED01499159919E01240F54
:108FE000351FE217F30771F480819181840F951F7B
:108FF000029611969C938E938281938113969C93F3
:109000008E931297E0E0F0E0D80112968D919C913A
:109010001397009719F0F8018C01F6CF8D919C9170
:1090200098012E5F3F4F820F931F2091E60C3091E5
:10903000E70C2817390769F4309729F41092E90CE6
:109040001092E80C02C0138212821093E70C009376
:10905000E60CDF91CF911F910F9108956627772736
:1090600009C244EE5CE000C0FA01A191B081009712
:1090700019F41097E1F0CD01DC01CD010D90002035
:1090800011F4C00113C0FB012191222319F0201516
:10909000D9F7F3CFFB012191201519F41E921196F7
:1090A00006C02223C1F70D900020A1F7D001FA01DC
:1090B000A193B0830895BB274A3031F4992322F459
:1090C000BDE2909581959F4F30C0BB272A3051F467
:1090D000992342F4BDE290958095709561957F4FFC
:1090E0008F4F9F4F01C0BB27FA01A62F6217710552
:1090F00081059105330B30FB66F0AA27660F771FB9
:10910000881F991FAA1FA21710F0A21B6395385041
:10911000A9F7A05DAA3308F0A95DA19336F7B111B4
:10912000B1931082CA0104C4BB27FB015527AA27AB
:10913000880F991FAA1FA41710F0A41B83955051E4
:10914000B9F7A05DAA3308F0A95DA193009779F75C
:10915000B111B1931192CB01EBC34F925F926F9219
:109160007F929F92AF92BF92CF92DF92EF92FF9247
:109170000F931F93CF93DF93CDB7DEB729970FB629
:10918000F894DEBF0FBECDBF6A01122FB02E2BE3C5
:10919000201720F0FF24F394F00E02C0BCE3FB2E56
:1091A0000F2D27E0AE014F5F5F4FCAD2AC0189811E
:1091B000982F9970913031F0E1FC06C0E0FE06C0B6
:1091C00090E205C09DE203C09BE201C090E0EE2D5D
:1091D000E07183FF3CC0911102C083E001C084E0D4
:1091E000811718F4212F281B01C020E0E1110BC0CA
:1091F000F601822F30E2882319F031938150FBCFA2
:10920000C20ED11C20E0992329F0D6019C93F601CF
:1092100031966F01C6010396E2FE0AC03EE4D60114
:109220003C9341E411964C93119712963C9306C0DF
:109230003EE6F601308341E641833283FC01322F62
:1092400040E2332309F442C041933150FACF82FF08
:1092500044C0911102C083E001C084E0811718F47A
:10926000212F281B01C020E0E1110BC0F601822F45
:1092700030E2882319F031938150FBCFC20ED11C0C
:1092800020E0992329F0D6019C93F60131966F01D5
:10929000C6010396E2FE0BC039E4D6013C933EE4DE
:1092A00011963C93119736E412963C9307C039E629
:1092B000F60130833EE6318336E63283FC01322FFD
:1092C00040E2332319F041933150FBCFFC01E20F10
:1092D000F11D10828EEF9FEFB7C0F1E0911101C038
:1092E000F0E06F2F70E01416150624F49A012F5F3A
:1092F0003F4F02C021E030E0260F371FBB2029F08E
:109300006B2D70E06F5F7F4F02C060E070E0260F52
:10931000371F612F70E0261737071CF4121B212F0F
:1093200001C020E03E2D387159F4D601322F60E2A1
:10933000332319F06D933150FBCFC20ED11C20E0C6
:10934000FF2331F0D6019C93B6016F5F7F4F6B0115
:10935000E1110BC0F601922F30E3992319F03193FC
:109360009150FBCFC20ED11C20E09F2D940F3A816B
:10937000782F7071A72E84FF03C0313309F4915008
:10938000191624F4993018F098E001C091E0E42F08
:10939000852F57FF02C0E0E080E06E2F782FE0E0DD
:1093A000F0E0AEE29A2E3A01691A71082A01461AD3
:1093B000570A0B2D10E01195019511096F3F8FEFA2
:1093C000780729F4D6019C92C60101966C014617D4
:1093D000570784F0661677066CF47F01E40CF51CE1
:1093E000A1E0B0E0AC0FBD1FEA0EFB1ED701119645
:1093F000BC9002C090E3B92E615071093196C6014C
:1094000001967C016017710724F0D601BC926C01B3
:10941000D5CF6417750741F4363320F4353321F482
:10942000A11002C081E3B82EF601B082F701822FAD
:1094300090E2882319F091938150FBCFF701E20F5E
:10944000F11D108280E090E029960FB6F894DEBFFF
:109450000FBECDBFDF91CF911F910F91FF90EF9085
:10946000DF90CF90BF90AF909F907F906F905F9074
:109470004F9008956F927F928F929F92AF92BF927A
:10948000CF92DF92EF92FF920F931F93CF93DF93D0
:10949000EC017B016115710519F0DB018D939C9343
:1094A0008E010F5F1F4F7880872D90E021D2892B8E
:1094B00011F0E801F5CFBDE27B1205C00F5F1F4F31
:1094C0007980C1E008C0EBE27E1204C08E010E5F1D
:1094D0001F4F7980C0E06801F1E0CF1AD10843E066
:1094E00050E064EF72E0C6010BD2892BE9F4680109
:1094F00022E0C20ED11C45E050E06FEE72E0C601E2
:10950000FFD1892B21F4680187E0C80ED11CE1143A
:10951000F10419F0D701CD92DC92C111F9C060E0DD
:1095200070E080E89FE7FDC043E050E06CEE72E041
:10953000C601E6D1892B51F4E114F10409F4EDC020
:109540000E5F1F4FF70111830083E7C0680160E0E1
:1095500070E0CB0100E010E0F601D0EDD70DDA307D
:1095600050F52C2F2260622E2C2F2870C2FF05C0D0
:10957000211127C00F5F1F4F24C0222311F001507B
:109580001109A5E0B0E09B01AC0130D34B015C01B7
:10959000880C991CAA1CBB1CC501B4016D0F711D60
:1095A000811D911D6839A9E97A078A07A9E19A07FF
:1095B00040F0C66005C0DE3F51F4C3FD44C0C86042
:1095C0006C2EBFEFCB1ADB0A7080C62DC5CF2D2FB6
:1095D0002F7D2531C1F540814D3211F4C06106C0A7
:1095E0004B3221F0319621E030E006C03296D601B0
:1095F00011964C9122E030E0A0EDA40FAA3018F0B3
:10960000E21BF30B20C040E050E04038BCE05B07B9
:109610005CF49A01220F331F220F331F420F531F96
:10962000440F551F4A0F511D3196DF0111972C91A0
:10963000A0EDA20FAA3048F3C4FF03C05195419595
:109640005109040F151FC1FF07C0E114F10421F0F7
:109650003197D701ED93FC937FD1C370C33019F0DC
:109660006B017C0106C06B017C01F7FAF094F7F8FE
:10967000F09420E030E0A901C701B60169D1882348
:1096800009F443C017FF06C0119501951109CBE0FD
:10969000D3E002C0C3E2D3E05E01B8E1AB1AB10887
:1096A0004601BE2DAF2D90E2E92EF12C0E151F05BF
:1096B0007CF0FE012591359145915491B4018B2F99
:1096C0009A2FABD14B01B82FA92F0E191F09EECF3E
:1096D0002497F594E794CA15DB0541F76401EB2E56
:1096E000FA2E8E2D880F8F2D881F8F3F41F020E09E
:1096F00030E0A901C701B6012BD1811106C082E279
:1097000090E09093EB0C8093EA0CC701B60109C07E
:1097100060E070E080E89FEF04C060E070E080EC03
:109720009FE7DF91CF911F910F91FF90EF90DF9016
:10973000CF90BF90AF909F908F907F906F90089543
:10974000283008F027E03327DA01990F311D87FD13
:10975000916000966105710539F432602E5F3D938A
:1097600030E32A95E1F708959F3F30F08038710586
:10977000610509F03C5F3C5F3D93913008F08068E3
:10978000911DDF93CF931F930F93FF92EF92192FA9
:10979000987F9695E92F96959695E90FFF27EF57B5
:1097A000FC4F99273327EE24FF24A701E7010590FA
:1097B0000894079428F4360FE71EF81E491F511D20
:1097C000660F771F881F991F0694A1F705900794CD
:1097D00028F4E70EF81E491F561FC11D770F881F7A
:1097E000991F661F0694A1F70590079428F4F80EB8
:1097F000491F561FC71FD11D880F991F661F771F4E
:109800000694A1F70590079420F4490F561FC71F2F
:10981000D81F990F661F771F881F0694A9F7849198
:109820001095177041F0D695C79557954795F794C1
:10983000E7941A95C1F7E7E2F3E068941590159163
:1098400035916591959105907FE27395E118F10A44
:10985000430B560BC90BD009C0F7E10CF11E431F97
:10986000561FC91FD01D7EF4703311F48A95E6CFC0
:10987000E894015030F0080F0AF40027021708F4AA
:10988000202F2395022F7A3328F079E37D932A95B0
:10989000E9F710C07D932A9589F606949795679508
:1098A000379517951794E118F10A430B560BC90B1E
:1098B000D00998F023957E9173957A3308F070E380
:1098C0007C932013B8F77E9170617D9330F083957F
:1098D00071E37D9370E32A95E1F71124EF90FF90F7
:1098E0000F911F91CF91DF91992787FD9095089552
:1098F0009111F6C0803219F089508550D0F7089543
:10990000FB01DC014150504088F08D9181341CF006
:109910008B350CF4805E659161341CF06B350CF472
:10992000605E861B611171F3990B0895881BFCCF53
:10993000DC01FC01672F71917723E1F7329704C0B6
:109940007C916D9370836291AE17BF07C8F3089541
:1099500040D008F481E00895E89409C097FB3EF4F4
:1099600090958095709561957F4F8F4F9F4F99236C
:10997000A9F0F92F96E9BB279395F69587957795EA
:109980006795B795F111F8CFFAF4BB0F11F460FFAA
:109990001BC06F5F7F4F8F4F9F4F16C0882311F002
:1099A00096E911C0772321F09EE8872F762F05C016
:1099B000662371F096E8862F70E060E02AF09A95B1
:1099C000660F771F881FDAF7880F9695879597F9A6
:1099D0000895990F0008550FAA0BE0E8FEEF161640
:1099E0001706E807F907C0F012161306E407F50793
:1099F00098F0621B730B840B950B39F40A2661F007
:109A0000232B242B252B21F408950A2609F4A140A9
:109A1000A6958FEF811D811D08950BD07BC06CD062
:109A200028F071D018F0952309F05DC062C01124B0
:109A3000A5C081D0A0F3959FD1F3950F50E0551F9D
:109A4000629FF001729FBB27F00DB11D639FAA2793
:109A5000F00DB11DAA1F649F6627B00DA11D661FE2
:109A6000829F2227B00DA11D621F739FB00DA11D03
:109A7000621F839FA00D611D221F749F3327A00DBD
:109A8000611D231F849F600D211D822F762F6A2F59
:109A900011249F5750408AF0E1F088234AF0EE0FDE
:109AA000FF1FBB1F661F771F881F91505040A9F7EB
:109AB0009E3F510570F017C061C05F3FECF3983EC8
:109AC000DCF3869577956795B795F795E7959F5F52
:109AD000C1F7FE2B880F911D9695879597F90895EC
:109AE00099278827089597F99F6780E870E060E0DC
:109AF00008959FEF80EC089500240A941616170627
:109B000018060906089500240A941216130614066E
:109B100005060895092E0394000C11F4882352F0D1
:109B2000BB0F40F4BF2B11F460FF04C06F5F7F4F89
:109B30008F4F9F4F089557FD9058440F551F59F070
:109B40005F3F71F04795880F97FB991F61F09F3F2A
:109B500079F087950895121613061406551FF2CF53
:109B60004695F1DF08C0161617061806991FF1CFA3
:109B700086957105610508940895E894BB276627CA
:109B80007727CB0197F90895F999FECF92BD81BD52
:109B9000F89A992780B50895262FF999FECF1FBA14
:109BA00092BD81BD20BD0FB6F894FA9AF99A0FBE06
:109BB00001960895052E97FB16F400940FD057FDDB
:109BC00005D024D007FC02D046F408C0509540953B
:109BD000309521953F4F4F4F5F4F08959095809559
:109BE000709561957F4F8F4F9F4F089531D0A59FFE
:109BF000900DB49F900DA49F800D911D1124089588
:109C0000B7FFF4CFF3DF821B930B0895A1E21A2E66
:109C1000AA1BBB1BFD010DC0AA1FBB1FEE1FFF1F10
:109C2000A217B307E407F50720F0A21BB30BE40B60
:109C3000F50B661F771F881F991F1A9469F76095A7
:109C40007095809590959B01AC01BD01CF01089561
:109C5000A29FB001B39FC001A39F700D811D11246D
:109C6000911DB29F700D811D1124911D08955058B2
:109C7000BB27AA270ED04ECF3FDF30F044DF20F0C5
:109C800031F49F3F11F41EF434CF0EF4E095E7FB5E
:109C90002ACFE92F50DF80F3BA17620773078407D2
:109CA000950718F071F49EF568CF0EF4E0950B2E31
:109CB000BA2FA02D0B01B90190010C01CA01A0011E
:109CC0001124FF27591B99F0593F50F4503E68F179
:109CD0001A16F040A22F232F342F4427585FF3CFBA
:109CE000469537952795A795F0405395C9F77EF48B
:109CF0001F16BA0B620B730B840BBAF09150A1F0D4
:109D0000FF0FBB1F661F771F881FC2F70EC0BA0F59
:109D1000621F731F841F48F4879577956795B795E1
:109D2000F7959E3F08F0B3CF9395880F08F09927D9
:109D3000EE0F9795879508950CD0ECCEE4DE40F0B9
:109D4000DBDE30F021F45F3F19F0CDCE511116CF9C
:109D5000D0CEF1DE98F39923C9F35523B1F3951BC7
:109D6000550BBB27AA2762177307840738F09F5F3C
:109D70005F4F220F331F441FAA1FA9F333D00E2EAB
:109D80003AF0E0E830D091505040E695001CCAF718
:109D900029D0FE2F27D0660F771F881FBB1F2617DD
:109DA00037074807AB07B0E809F0BB0B802DBF01B0
:109DB000FF2793585F4F2AF09E3F510568F093CEDE
:109DC000DDCE5F3FECF3983EDCF3869577956795A3
:109DD000B795F7959F5FC9F7880F911D9695879561
:109DE00097F90895E1E0660F771F881FBB1F621780
:109DF00073078407BA0720F0621B730B840BBA0B3E
:109E0000EE1F88F7E095089504D06894B111B6CE9E
:109E1000089599DE88F09F5790F0B92F9927B75190
:109E2000A0F0D1F0660F771F881F991F1AF0BA951E
:109E3000C9F712C0B13081F0A0DEB1E008959DCE27
:109E4000672F782F8827B85F39F0B93FCCF3869514
:109E500077956795B395D9F73EF490958095709571
:109E600061957F4F8F4F9F4F0895B3DD08F48FEFBB
:109E70000895AFDD880B990B0895EE0FFF1F881F23
:109E80008BBF0790F691E02D19946F927F928F927D
:109E90009F92AF92BF92CF92DF92EF92FF920F9379
:109EA0001F93CF93DF93EC01009789F4CB01DF91EF
:109EB000CF911F910F91FF90EF90DF90CF90BF90C7
:109EC000AF909F908F907F906F900C940147FC0112
:109ED000E60FF71F9C0122503109E217F30708F43F
:109EE000AAC0D9010D911C91119706171707A8F068
:109EF0000530110508F49DC0C8010497861797071F
:109F000008F497C002501109061B170B0193119317
:109F10006D937C93CF010AD88CC05B01A01AB10A63
:109F20004C01800E911EA091E80CB091E90C40E02C
:109F300050E0E12CF12C109709F44AC0A815B9059E
:109F4000D1F56D907C901197630182E0C80ED11C11
:109F5000CA14DB0480F1A3014A195B096A0182E09B
:109F6000C80ED11C1296BC9012971396AC91B5E016
:109F7000CB16D10440F0B282A38351834083D90130
:109F80006D937C930AC00E5F1F4FC301800F911F1A
:109F9000F90191838083EB2DFA2FE114F10431F064
:109FA000D7011396FC93EE93129743C0F093E90CFC
:109FB000E093E80C3EC08D919C911197481759078A
:109FC00008F4AC017D0112960D90BC91A02DB3CF89
:109FD0008091E60C9091E70C88159905E1F44617FD
:109FE0005707C8F48091020290910302009741F450
:109FF0008DB79EB74091060250910702841B950BC6
:10A00000E817F907C0F4F093E70CE093E60CF901C8
:10A01000718360830EC0CB010E9401477C010097D1
:10A0200051F0A801BE011CD0CE010E949647C70185
:10A0300004C0CE0102C080E090E0DF91CF911F917B
:10A040000F91FF90EF90DF90CF90BF90AF909F90D7
:10A050008F907F906F90089581E090E0F89419C000
:10A06000FB01DC0102C001900D9241505040D8F735
:10A070000895FB01DC018D91019080190110D9F345
:10A08000990B0895FB01DC0101900D920020E1F78E
:10A09000089512E0C2EAD2E000E005C0802FFE0180
:10A0A000ECDE2196011DC33AD10780E00807B1F725
:04A0B000F894FFCF52
:10A0B400FFFF0000EC0C8000200A0D0000000000EF
:10A0C400004B178813F616000000004C178A13255E
:10A0D4001A00000000F1359A339E34000000005F3E
:10A0E4002DA72CD92C00000000992B36269A260087
:10A0F4000000009A0967075808000000004A358CE0
:10A10400339E3300000000F0359833D6330000004E
:10A1140000012B3826612600000000ED3592336DD6
:10A124003400000000EE32AB2C212D000000004B67
:10A13400358E330E3400000000F2359C332C35008C
:10A144000000004C359033013500000000EF3596D7
:10A154003316350000000049358A33C4340000004A
:10A16400005D2DA32CAD2C000000009809630707A7
:10A174000A00000000602DA92C0A2D00000000EE4A
:10A184003594339134000000005E2DA52C882C00FA
:10A1940000000099096507690752303300523032D4
:10A1A40000523037005230310052303900523838C2
:10A1B40000523837005238380052303000523837A5
:10A1C40000523038005231330052313200523131B2
:10A1D4000052373300523732005237310052313790
:10A1E40000523136005231350001000000010000F8
:10A1F4000001000000523835005238340052303526
:10A204000052303600362E342E302E4600005230A6
:10A21400340052383700000000001A258424B32487
:10A224006025E424C224D624000000004835883385
:10A234005239392041524455494E4F2053544152CA
:10A2440054555020434F4D504C4554450D0A002A57
:10A254000047300047303000473100473031004775
:10A264003238004630390046390046313100463133
:10A274003200463133004631340046313500463130
:10A284003600463230004632310046323200463320
:10A29400310046333200463431004634320046340D
:10A2A40033004634340046363100463831004638EF
:10A2B40032004638330046383400200A0D00523943
:10A2C400392068616E646C6572203D3D204E554CAA
:10A2D4004C0D0A0052393900207265736574746933
:10A2E4006E67206469676974616C2070696E002010
:10A2F400726573657474696E6720616E616C6F67F3
:10A304002070696E0052393920484F4D45205A203B
:10A314004F4E20535441525455500D0A005239396E
:10A3240020484F4D452059204F4E205354415254FC
:10A3340055500D0A0052393920484F4D45205820B8
:10A344004F4E20535441525455500D0A005239393E
:10A354002057696C6C207A65726F20580052393925
:10A364002057696C6C207A65726F20590052393914
:10A374002057696C6C207A65726F205A0052323112
:10A384000050005600523939204572726F723A20DB
:10A39400696E76616C696420706172616D65746563
:10A3A400722069640D0A0052343100686F6D650DC6
:10A3B4000A0052393920656D657267656E637920CC
:10A3C40073746F700D0A00523939206572726F729E
:10A3D4000D0A00523832005239392073746F70708C
:10A3E40065640D0A00523939206572726F7220005B
:10A3F4002064656163746976617465206D6F746F40
:10A404007220582064756520746F206D69737365BC
:10A414006420737465707300206465616374697685
:10A42400617465206D6F746F7220592064756520A6
:10A43400746F206D69737365642073746570730041
:10A444002064656163746976617465206D6F746FEF
:10A4540072205A2064756520746F206D697373656A
:10A4640064207374657073005239392074696D65A2
:10A474006F7574205820617869730D0A0052393958
:10A484002074696D656F7574205920617869730D46
:10A494000A005239392074696D656F7574205A2029
:10A4A400617869730D0A0020510052383100205838
:10A4B4004100205842002059410020594200205AAE
:10A4C4004100205A42002073746120002063757299
:10A4D400200020656E6420002068616C66200020E6
:10A4E4006C656E2000206D696E2000206D617820FF
:10A4F4000020737064200052323000523833200040
:10A504005239392043616C6962726174696F6E20DB
:10A514006572726F723A20696E76616C696420614B
:10A524007869732073656C65637465640D0A002033
:10A534006178697320002061742073746172746996
:10A544006E6720706F696E7400523233002063614D
:10A554006C6962726174696E67206C656E67746899
:10A5640000207374657020636F756E743A20005216
:10A574003939206D6F76656D656E7420646F6E6514
:10A584000D0A0020617420656E6420706F696E741A
:10A59400005239392043616C6962726174696F6E6B
:10A5A400206572726F723A20656E642073746F70E6
:10A5B40020616374697665206265666F72652073D5
:10A5C400746172740D0A00206D6F766520746F20BB
:10A5D400737461727420666F722063616C69627255
:10A5E4006174696F6E006E616E00696E66006F76ED
:02A5F4006600FF
:00000001FF
